:1000000000800020BD010000614300002543000086
:100010002543000025430000254300002543000040
:1000200025430000254300002543000061430000F4
:1000300061430000254300006143000015430000B8
:100040006143000061430000614300006143000020
:100050006143000061430000614300006143000010
:100060006143000061430000614300006143000000
:1000700061430000614300006143000061430000F0
:1000800061430000614300006143000061430000E0
:1000900061430000614300006143000061430000D0
:1000A000753C0000614300006143000061430000B3
:1000B00061430000614300006143000061430000B0
:1000C00061430000614300006143000061430000A0
:1000D0006143000061430000614300006143000090
:1000E0006143000061430000614300006143000080
:1000F00061430000256300006143000021690000A6
:1001000061430000416E0000614300006143000054
:10011000614300006143000061430000614300004F
:10012000614300006143000061430000614300003F
:10013000614300006143000061430000614300002F
:10014000614300006143000061430000614300001F
:10015000614300006143000061430000614300000F
:1001600061430000154B0000614300006143000043
:1001700061430000614300006143000061430000EF
:1001800061430000614300006143000061430000DF
:1001900061430000614300006143000061430000CF
:1001A00061430000614300006143000061430000BF
:1001B0006143000061430000E5570000574B4CF2DB
:1001C000205210B51A804DF628121A8000BF00BFC9
:1001D00004F0CAF8524B4FF010621A60514A9A600C
:1001E000514ADA60A3F53043203B1A6812F480725A
:1001F00004D14E490A604FF4A8521A604C4B1A7849
:10020000110703D51A7842F008021A70494B4A4C7C
:100210004A482A221A704A4A00239918A14203D256
:10022000195899500433F8E7464B474900228B424E
:1002300002D243F8042BFAE74448454900235A58B0
:100240001A500433B3F5DE7FF9D1424B424A802184
:1002500003F8011B9342FBD1404B3C4A1A60404BD0
:100260000A221A70A3F5805324225A70A0221A7011
:100270009A799207FCD59A79D406FCD4394A9379B5
:1002800003F00C03082B374BF9D105221A714322D6
:100290005A719A799006FCD5324A9179314B4906C8
:1002A000FBD5314A4FF08171116005215160202248
:1002B0001A709A7902F00C020C2AFAD12B4B2C4AB4
:1002C0001A602C4B2C4A1A6000225A60072243F80D
:1002D000042C2A4AC3F80C2D62B604F0DDFA134B45
:1002E0001B68DA0705D5264804F038FA254B264A5C
:1002F0001A60264B1B785B0609D5224C224A2368DC
:10030000934204D11E4804F029FA0023236009F027
:1003100077F804F02FF805F005FDFEE70E20054004
:1003200030800440823F04000100002B14D00340C1
:1003300002D0074000E007409098FF1F9CB70000E4
:10034000608FFF1F9098FF1F94FFFF1F008AFF1F01
:100350000000000000E400E05FE400E008ED00E0E1
:1003600000500640004006404480044004800440A1
:10037000C010050014E000E03F190100000020203B
:100380007AFBF2561CE00340A5C3945A00F00740E4
:10039000FFFFFFFFFFFFFFFFFFFFFFFFFFFFFFFF6D
:1003A000FFFFFFFFFFFFFFFFFFFFFFFFFFFFFFFF5D
:1003B000FFFFFFFFFFFFFFFFFFFFFFFFFFFFFFFF4D
:1003C000FFFFFFFFFFFFFFFFFFFFFFFFFFFFFFFF3D
:1003D000FFFFFFFFFFFFFFFFFFFFFFFFFFFFFFFF2D
:1003E000FFFFFFFFFFFFFFFFFFFFFFFFFFFFFFFF1D
:1003F000FFFFFFFFFFFFFFFFFFFFFFFFFFFFFFFF0D
:10040000FFFFFFFFFFFFFFFFFFFFFFFFFEFFFFFFFD
:1004100010B5054C237833B9044B13B10448AFF33E
:1004200000800123237010BD9098FF1F0000000082
:100430009CB7000008B5064B1BB106480649AFF350
:1004400000800648036813B1054B03B1984708BD07
:10045000000000009CB700009498FF1F9098FF1FB9
:10046000000000000122014B1A707047909AFF1F94
:1004700008B505F0C1FB08BD10B50446034A40F8B5
:100480001C2B01F0A7FD204610BD00BFA0B200004C
:1004900038B5064D05F5BB442C34143D204605F017
:1004A000CFFA143CAC42F9D138BD00BFC09AFF1F4F
:1004B00010B5074C23685B68204606490E22984712
:1004C000204605F059FA044A044B1A6010BD00BFDB
:1004D00078FDFF1F78AE00000400FA050CED00E087
:1004E0000F4B03604172026100230372C36039B194
:1004F0001946026942F823100133427A9A42F8DC25
:10050000084B1A680AB9186004E053690BB11A461F
:10051000FBE75061002343618380C380704700BFC5
:1005200070AE000048FDFF1F2DE9F04FA3B0064656
:1005300001915F4FDFF894B106A83146012201F026
:1005400089FF06A801F09AFD002800F0A38006A804
:1005500001F046FD014602A805F0BEFA02A83946A0
:1005600005F0A8FB00283CD00EA8524905F0B4FACB
:1005700002A80EA905F092FB04460EA805F060FA49
:100580007CBB584605F0C6FB04464B4B1B689842A3
:10059000C4BF494B1860DFF83881484D55F820300A
:1005A00003EB830340F2DC5909FB00F909EB830AF2
:1005B000C24406A801F014FD0146504605F0B6FA03
:1005C00055F824A006A801F033FD0AEB8A0A09EBCE
:1005D0008A09C844C8F8100055F82430013345F89A
:1005E000243006A801F0FEFC002857D012A8344998
:1005F00005F072FA02A812A905F050FB00284FD1AD
:1006000016A8304905F068FA02A816A905F046FBBD
:10061000D0F1010438BF002416A805F011FA00E05B
:10062000002412A805F00CFA54B306A801F0D8FC77
:100630000146584605F07AFA9DF81C308DF86C306A
:10064000089B1C939DF824308DF874301E4B1A9330
:1006500022AB53F8630D59689A68CDF87500CDF850
:100660007910CDF87D201B7B8DF881300D9B219377
:100670001AA8019B591CFFF757FF1AA801F0AAFC02
:1006800006A801F0EFFC02A805F0DAF906A801F0CF
:10069000A1FC51E706A801F09DFC06E0002300E064
:1006A0000123002BBCD10024BEE723B0BDE8F08FAE
:1006B0001C9AFF1F88AE00003C9AFF1F489AFF1F3C
:1006C0008CAE000094AE0000E0B20000E099FF1F85
:1006D000C09AFF1F30B585B004460D4668462146D6
:1006E0000A2205F035FA68460E4905F061FA05EB75
:1006F000850540F2DC5303FB04F404EB85056846F2
:100700000949294405F04CFA084C68462146112253
:10071000002305F0E7FA684605F092F9204605B097
:1007200030BD00BF9CAE0000C09AFF1F009AFF1FA3
:1007300038B5164C23685B68204615490522984752
:100740002046144B196805F063F923685B6820465E
:100750001149092298472046104B196805F058F9AD
:1007600023685B6820460E49062298470D4B1D689A
:1007700028460AF08FF8024623685B68204629461F
:100780009847204605F0F8F838BD00BF78FDFF1FF8
:10079000A4AE00000099FF1FACAE0000149AFF1F2A
:1007A000B8AE0000BC99FF1F10B504460620C4F384
:1007B000C00103F0E3FF0520C4F3800103F0DEFF76
:1007C0000420C4F3400103F0D9FF032004F0010129
:1007D00003F0D4FF10BD00BF38B572B62F4B1B7F9E
:1007E00003F0FF0213B100212C4B197762B6002AE7
:1007F00052D02B4B1A682B4B1A6072B6274BB3F9A9
:100800002000B3F91E20801A47F6FF72DA834FF4F6
:1008100000421A8462B608F099FB234908F09EFC56
:100820004FF0814108F0E6FB0446002108F094FDFA
:1008300038B120464FF07C5108F0D4FA08F0A0FD02
:1008400006E020464FF07C5108F0CAFA08F098FD07
:1008500007F09AFF02460B4600204FF0804106F059
:1008600069FD04460D460022002308F079FA40B1E4
:100870002046294600220D4B07F03AFE08F084FA84
:1008800007E0204629460022084B07F02FFE08F01B
:100890007BFA0138FFF788FF38BD00BF0C99FF1FB6
:1008A00050FCFF1FBC9AFF1F00FF7F470000E03F86
:1008B00008B505F02FFA012814BF0020012008BD5B
:1008C00030B5A1B004460D46544905F0B1F958B110
:1008D0006846294605F01EF96846FFF7E9FF504BC8
:1008E0001870684605F0ACF820464E4905F0A0F9AE
:1008F00020B1284605F00EFA4B4B186020464B49B4
:1009000005F096F958B104A8294605F003F904A8A2
:10091000FFF7CEFF464B187004A805F091F820466B
:10092000444905F085F920B1284605F0F3F9424B1A
:1009300018602046414905F07BF958B108A82946BE
:1009400005F0E8F808A8FFF7B3FF3D4B187008A8BA
:1009500005F076F820463B4905F06AF958B10CA835
:10096000294605F0D7F80CA8FFF7A2FF364B187000
:100970000CA805F065F82046344905F059F958B13E
:1009800010A8294605F0C6F810A8FFF791FF304BD4
:10099000187010A805F054F820462E4905F048F9C3
:1009A00058B114A8294605F0B5F814A8FFF780FF40
:1009B000294B187014A805F043F82046274905F084
:1009C00037F920B1284605F0A5F9254B18602046D7
:1009D000244905F02DF958B118A8294605F09AF8D0
:1009E00018A8FFF765FF204B187018A805F028F825
:1009F00020461E4905F01CF970B11CA8294605F0D7
:100A000089F81CA8FFF754FF194B18701CA805F0B3
:100A100017F80122174B1A7021B030BD60AF0000EB
:100A2000F899FF1F68AF0000748FFF1F70AF0000C0
:100A3000788FFF1F7CAF00006C8FFF1F88AF000016
:100A4000808FFF1F9CAF0000708FFF1FACAF0000B6
:100A5000F099FF1FC0AF00008C99FF1FD4AF0000BA
:100A6000848FFF1FE4AF0000888FFF1FECAF0000F2
:100A7000698FFF1F889AFF1F30B5A1B0684600211B
:100A800005F02AF804A8002105F026F808A849492D
:100A9000494A012301F048FC484C9DF82430237159
:100AA0000A9BA3609DF82C30237320AB53F8535D51
:100AB00058689968C4F80D50C4F81100C4F81510AE
:100AC0001B7B63760F9BE36108A801F083FA204645
:100AD00001F0D4FA00285BD0254650E0284601F00A
:100AE00003FAC4B23D2C14D010A8694605F012F8E0
:100AF00010A8214605F07AF80146684605F000F88E
:100B000010A804F09DFF284601F0EEF9C4B23D2C78
:100B1000EAD1284601F0E8F9C4B20A2C2FD014A873
:100B200004A904F0F7FF14A8214605F05FF8014678
:100B300004A804F0E5FF14A804F082FF284601F0A1
:100B4000D3F9C4B20A2CEAD118A8694604F0E2FF2E
:100B50001CA804A904F0DEFF18A81CA9FFF7B0FE2A
:100B60001CA804F06DFF18A804F06AFF144C684636
:100B7000214604F0DBFF04A8214604F0D7FF2846F5
:100B800001F05CFA0028A9D10C4801F06BFA09E0E9
:100B90000C4C23685B6820460B491A229847204674
:100BA00004F0EAFE04A804F04BFF684604F048FF96
:100BB00021B030BDE0F8FF1FF4AF0000E098FF1F48
:100BC000F4AE000078FDFF1F04B0000030B589B01E
:100BD000624D634C2846214601F030FC68462946A8
:100BE0002246132301F0A0FB5E4C9DF804302371D4
:100BF000029BA3609DF80C30237308AB53F8135D80
:100C000058689968C4F80D50C4F81100C4F815105C
:100C10001B7B6376079BE361684601F0DBF9236881
:100C20005B68204650490522984720464F4B19786B
:100C300004F0EEFE204604F09FFE23685B68204629
:100C40004B490822984720464A4B196804F0E0FEB9
:100C5000204604F091FE23685B68204646490A223C
:100C600098472046454B197804F0D2FE204604F000
:100C700083FE23685B68204641490A229847204644
:100C8000404B196804F0C4FE204604F075FE23684A
:100C90005B6820463C491122984720463B4B197817
:100CA00004F0B6FE204604F067FE23685B68204629
:100CB0003749102298472046364B197804F0A8FE91
:100CC000204604F059FE23685B6820463249122210
:100CD00098472046314B197804F09AFE204604F0DC
:100CE0004BFE23685B6820462D4911229847204619
:100CF0002C4B197804F08CFE204604F03DFE23684E
:100D00005B68204628490F2298472046274B1968E0
:100D100004F07EFE204604F02FFE23685B68204628
:100D20002349082298472046224B197804F070FE88
:100D3000204604F021FE23685B6820461E490522F8
:100D4000984720461D4B197804F062FE204604F0B7
:100D500013FE204601F086F909B030BDE0F8FF1F10
:100D6000F4AF0000E098FF1FE4AE0000F899FF1F09
:100D7000ECAE0000748FFF1FF8AE0000788FFF1FED
:100D800004AF00006C8FFF1F10AF0000808FFF1FAB
:100D900024AF0000708FFF1F38AF0000F099FF1FD5
:100DA0004CAF00008C99FF1F20B00000848FFF1F04
:100DB00030B00000888FFF1F3CB00000698FFF1F1C
:100DC0002DE9F04192B00220002103F009FD082036
:100DD000002103F005FD0920002103F001FD0B2097
:100DE000012103F0FDFC0620012103F0F9FC0520A0
:100DF000012103F0F5FC0420012103F0F1FC0320A4
:100E0000012103F0EDFC684B1868FFF7CDFC674843
:100E1000052104F0C7FB664B1A7842F005021A70F0
:100E200064480A2101F0E0F9F0B90024614D624FF5
:100E3000624E13E00F20FFF7B7FC642003F016FDAD
:100E40000020FFF7B1FC642003F010FD0134062CF4
:100E500004DD4FF4FA7003F009FD3E6028460A21D4
:100E600001F0C2F90028E5D0524D02A82946544AA3
:100E7000012301F059FA534B9DF80C201A71049A82
:100E80009A609DF814201A7312AA52F8336D5068B4
:100E90009168C3F80D60C3F81100C3F81510127BF8
:100EA0005A76099ADA6102A801F094F82846464970
:100EB00001F0B8FA40B1FFF7DFFD444B1B782BB9C6
:100EC0000022434B1A7001E0FFF780FE3D4B1A7978
:100ED0008DF82C209A680C921A7B8DF834203D4AAC
:100EE0000A921A4652F80D4F50689168CDF8354075
:100EF000CDF83900CDF83D10127B8DF84120DB692B
:100F000011930AA80021FFF70FFB0AA801F062F86D
:100F10002F4B1B789BB1304E341F304D3C36DFF8E1
:100F2000E480142754F8041F002904DD28463A46BB
:100F3000434608F01BFE05F2DC55B442F2D1002016
:100F400003F0BCF9264B1B68984205DC164B186071
:100F50000122244B1A7003E00020014603F0C2F97D
:100F6000214A224B9A6109202149032203F096FB72
:100F7000204803685B6820490A2298471F4B1B687A
:100F800023B91F4B12AAD31A019302E001AAD31A64
:100F90000193184C2046019904F03AFD204604F0D4
:100FA000EBFC12B0BDE8F0810099FF1F0082FF1F2B
:100FB00074FDFF1FE0F8FF1F0CED00E00400FA05D0
:100FC0009CAE0000AC98FF1FF4AF0000889AFF1F92
:100FD000698FFF1FE0B20000489AFF1FC09AFF1FF1
:100FE0003C9AFF1F688FFF1FB10400004499FF1F48
:100FF0006504000078FDFF1F44B00000A08FFF1FB4
:10100000D8FFFF1F710400002DE9F04F87B0954B0A
:101010001B68002B20DD0026354634463746B04697
:101020004FF0170B4FF0140ADFF83892584603F0D0
:1010300061F88044504603F05DF80744152003F042
:1010400059F80444162003F055F805440136D9F840
:101050000030B342EADC03E000252C462F46A846C8
:1010600098FBF3F897FBF3F794FBF3F495FBF3F598
:101070007D4B1E68B442B8BF0024B542B8BF0025FE
:101080007A4B1B6804937A4BD3F800B0794B1B68FA
:101090000593794B1B68E31A83EAE372A2EBE372D0
:1010A0000292764B1B68EB1A83EAE37CACEBE37CA1
:1010B000CDF80CC008EB070040F2FF394845A8BF47
:1010C0004846DFF800A2DAF800206D4B53F82230D2
:1010D000009320EAE07000214FF480620B4604F098
:1010E000A1FC684B1968684B1B68DAF8002003EB19
:1010F000830E40F2DC5C0CFB02F202EB8E02DFF8A6
:10110000D0E17244D2F810E0604AA2FB0EC2C2EBFA
:101110000E0E02EB5E0E4FEA5E2E01FB0EFE621912
:101120004A4528BF4A46B2FBF1F909FB0EF998423D
:101130001AD0049AC2EB0803002BB8BF5B425B4590
:1011400040F38480524B1860524B1A78524B1A70FD
:10115000464BC3F8008079E04D4B18604F4B1A782E
:101160004D4B1A70434B1F604B4B1B7813B1012240
:101170004B4B1A70029B9E4208DC4A4BC3F800900E
:10118000494B1A78494B1A703B4B1C60DDF80CC078
:10119000664508DC434BC3F80090454B1A78434B37
:1011A0001A70364B1D60434800F0D4FA18B141481C
:1011B00000F0B2FA20B9404B1B7813F0FF0F0BD0B0
:1011C000374B1B782BB1374BC3F800900022344BC0
:1011D0001A700122354B1A700022374B1A70374CA7
:1011E0002668374D2B68F61A082003F0EBFA2368BF
:1011F00006FB103028602368181AB0F5167F2ED928
:10120000304A1368013313602F4A1268934202DD9B
:1012100000222C4B1A602B4B1968194B53F82130C4
:101220001B4A1268934202DC013B194A13600122F7
:10123000194B1A70214B1868214A10601A68234B09
:101240001A600020C9B203F04DF808E0059ABB1AF5
:10125000002BB8BF5B429B45FFF67EAF84E707B02B
:10126000BDE8F08F948FFF1F7C8FFF1FD898FF1F62
:101270008C8FFF1FF499FF1FCC98FF1FDC98FF1F76
:10128000489AFF1F848FFF1F149AFF1F051040000C
:10129000449AFF1F808FFF1F688FFF1F708FFF1FF3
:1012A000D098FF1F0499FF1FF099FF1F3099FF1F6F
:1012B0008C99FF1F2C9AFF1F909AFF1F50FCFF1F55
:1012C00080F8FF1F0099FF1F3C9AFF1F0899FF1F1E
:1012D000C09AFF1F38B5684B93F8443013F0FF0FE6
:1012E00004D1664B1B78002B40F0B280644B1B7816
:1012F0001BB9644B1B78002B6ED0FFF719FA624BB9
:101300001B78ABB1614C2368C3EBC303C3EB8313FE
:1013100005335F4AA2FB0313DB085E484FF0FF3141
:10132000B1FBF3F1002200F0C3FA206803F09EFA4B
:10133000594C5A4B18682168FFF7CCF9584B186084
:101340002268584B1A604F4B1B783BB94B4B1B78AC
:1013500023B1494800F0CEFC534B1860524C23682F
:1013600023F00F032360514D2B685B6828465049DA
:101370000A229847284621680A22002304F00CFB21
:10138000284604F0F9FA3C48454B1968226800F0F9
:1013900045FC3D4B1B7893B13C4B1B68C3EBC3032F
:1013A000C3EB831305333A4AA2FB0313DB08394826
:1013B0004FF0FF31B1FBF3F1012200F079FA374B26
:1013C0001868FFF7F1F900232D4A13702D4A1370A6
:1013D000384B1A68384B1A60364B1A68374B1B6803
:1013E000D31A374A12689A4205D8FFF70DFE314BDF
:1013F0001A68324B1A602F4B1A68324B1B68D31A8B
:10140000314A12689A4203D22A4B1A682D4B1A604D
:10141000284C2168284B1B68C91A0B2009298CBF4E
:101420000021012103F0AAF92268284B1B68D31A76
:10143000532B1FD92268264B1B68D31A254A1268E2
:101440009A4217D2244B1B78A3B1FFF7C5F938BDD8
:10145000124B1868134B1968FFF73CF90146104B03
:1014600018600548002200F0D9FB124B1A68124B95
:101470001A603BE738BD00BF4499FF1F888FFF1FEC
:10148000688FFF1F3099FF1FF899FF1F748FFF1F90
:10149000CDCCCCCC949AFF1F449AFF1F0099FF1F1C
:1014A000BC99FF1F149AFF1F0499FF1F78FDFF1FAF
:1014B00050B0000050FCFF1FD498FF1F409AFF1F40
:1014C000908FFF1F8C9AFF1F648FFF1FBC9AFF1F16
:1014D0000899FF1F6C8FFF1F788FFF1F2DE9F843BE
:1014E00002F0B2FE614C204600F066FDDFF8C081DC
:1014F00020465F49424607F069FF5E4E30460021B4
:101500000A46FEF7EDFF30465B4B40F81C3B00F00F
:1015100053FD304600F05EFB30465849424607F026
:1015200055FF574F3846012107F12402FEF7D8FF37
:10153000544B3B604FF0FF33BB61534D28460121B4
:1015400005F11802FEF7CCFF504B2B6047F6FF73F6
:10155000EB834FF400432B84DFF89491484601213C
:1015600009F11802FEF7BCFF494BC9F800304846A4
:1015700000F03CFA47480660476000240472447259
:10158000C46004F001F944480760C0F80490047294
:101590004472C46004F0F8F8404806604560047284
:1015A0004472C46004F0F0F83D4C20463D4904F01C
:1015B00093FA20463C49424607F008FF3B4D05F2AE
:1015C000DC5705F5C74808F11C0800260BE020464B
:1015D000314604F081FA1434AC42F8D13D4607F2AA
:1015E000DC57474503D02C4605F2DC55EFE7304C7D
:1015F00000203049224607F0E9FE2F4D28462F49AA
:1016000004F06AFA28462849224607F0DFFE2C4DEE
:10161000284600F0D1FC28461549224607F0D6FEA0
:1016200028480821142200F065F8274802211422D6
:1016300000F060F8254B1968254A11601968254AA1
:1016400011601968244A11601968244A11601968E8
:10165000234A11601968234A11601968224A1160EF
:101660001A68224B1A60BDE8F88300BFE098FF1F9C
:10167000D51F00004499FF1FA0B2000079040000AC
:10168000949AFF1F80B200000C99FF1F70B20000F7
:1016900090B200003499FF1FC099FF1FD099FF1F1F
:1016A0001C9AFF1F5CB00000415A0000C09AFF1F47
:1016B000608FFF1F91040000E099FF1F60B00000E1
:1016C000AC98FF1F2C9AFF1FAC99FF1F50FCFF1F07
:1016D000189AFF1FFC99FF1F8C9AFF1FD498FF1FB9
:1016E00080F8FF1F409AFF1F0899FF1FBC9AFF1F39
:1016F0009099FF1F38B504460D4642600023836071
:10170000044B1B680360084603F05CF820736573A4
:10171000204638BD50FCFF1F007B704710B50446C3
:10172000407B03F04FF8237B83420CD0084B1A68B0
:101730002368D21A63689A4207D3054B1B6823605B
:101740002073012010BD002010BD002010BD00BF7F
:1017500050FCFF1F10B50446FFF7E0FF034620B121
:101760000023A3600123A37311E0A2686AB10949B1
:1017700008682168411A8A4207D8064B1B68236013
:101780000023A3600123A37301E00022A273184683
:1017900010BD00BF50FCFF1FF8B50646002103F046
:1017A000C3FF0746B8B1031D00F58275B6F91E40A8
:1017B000B6F9201033F9022B9442A8BF1446914287
:1017C000B8BF11469D42F5D8F483318401233377A5
:1017D000384603F073FFF8BD2DE9F04F83B0019058
:1017E00084693CB9002103F09FFF00285AD003F020
:1017F00065FF57E0B4F1FF3F0FD10198002103F0DE
:1018000093FF044600284DD001982146002203F0A2
:1018100075FF204603F052FF44E00198002103F0D9
:101820008FFF804600283DD0019BD3F81CC093F861
:10183000209000231D4F9B464FF0FF3A4E46200E4E
:10184000C4F30F2108EB0302B2F90450C1F5803E46
:1018500037F91090013037F9100001FB00F109FB56
:101860000E11091401FB05F1C913918026B1E24361
:10187000944506D2644407E0A44504D2CCEB0404AA
:1018800002E0544600E05C460233B3F5807FD6D1D7
:10189000019B9C6118464146002203F02FFF404601
:1018A00003F00CFF03B0BDE8F08F00BF64B0000090
:1018B00072B6836913B90123836105E0B3F1FF3F79
:1018C00004BF6FF001038361C16180F8202062B61C
:1018D000704700BF10B5044604F020F8204610BD44
:1018E00008B503480349044A07F070FD08BD00BF6E
:1018F00084F8FF1FD5180000608FFF1F08B503484C
:101900000349044A07F062FD08BD00BF8CF8FF1FC1
:10191000D5180000608FFF1F08B5002103F004FFF9
:101920000246A0B172B60A4B186810B91A6062B6C6
:1019300008BD084B1B681BB9064B1A6062B608BD90
:1019400003490B60034B1A6062B603F0B7FE08BD93
:10195000A4F8FF1F94F8FF1F38B51C4B1A681268D3
:1019600019791B4B19701B4B9A4206D2A3F5807450
:1019700004F5807304F5007402E0174B03F58074DE
:10198000164A106898B1021D47F6FF7532F9021B1E
:101990002944091123F8021B9C42F7D803F08EFE5C
:1019A0000F4B1A680D490A6000221A6005E040F2E8
:1019B000FF7223F8022B9C42FBD80A4B1B781BB109
:1019C0004FF08042084B1A6038BD00BF98F8FF1FE7
:1019D0001F8000401488FF1F1487FF1FA4F8FF1FFB
:1019E00094F8FF1FA0F8FF1F08E200E070B54F4811
:1019F000012103F035FF4E4B1A6842F480521A6001
:101A0000802203F5032303F6F5731A700024494E70
:101A100001253480284602F029FF0834A4B223B2FD
:101A2000B3F5006FF5D1444B1B6813F4800F16D04B
:101A3000424B1A6848F6A2731A409A420FD1404BA3
:101A40001A6840F22F339A4209D13E4B1B68012B92
:101A500005D13D4B1A6840F201139A4217D0364B1C
:101A60001A6842F480021A600122A3F59033303BD9
:101A70001A6040F22F32083B1A60043B48F6A3720A
:101A80001A60324A1A6040F2011210331A60274C71
:101A900023681A6800222E491960236802211971EF
:101AA0005A7101209871D87119725A729A72DA7249
:101AB0001A736FF0010159734FF0FF319973D973A5
:101AC00019691C4919611A755A75D98A4FF48071C0
:101AD000D9821A765A769A76DA76D88BD983998B08
:101AE00006219983237903F1804303F504331A70A7
:101AF000B0221A7003F060FE164B18702279164B54
:101B00001A70227902F110011448154B43F8210094
:101B100053119B0003F1604303F5614302F01F0280
:101B2000012101FA02F21A6070BD00BF98F8FF1F90
:101B30002C80044000C00C403C8004400060034006
:101B4000046003400C60034010600340A28F01005A
:101B50001487FF1FA0F8FF1F1B80004059190000C9
:101B6000008AFF1F08B503480349044A07F02EFC0A
:101B700008BD00BF98F8FF1FD5180000608FFF1F39
:101B800008B503480349044A07F020FC08BD00BF1C
:101B9000A8F8FF1FD5180000608FFF1F08B5034885
:101BA0000349044A07F012FC08BD00BFB0F8FF1F4C
:101BB000D5180000608FFF1F08B503480349044A89
:101BC00007F004FC08BD00BFB8F8FF1FD5180000DF
:101BD000608FFF1F002380F844300364C3637047A5
:101BE00008B572B690F8443013F0FF0F12D00023FE
:101BF00080F8443062B61C3000F034FA064B1B8883
:101C000023B1013B9BB2044A138023B95E2000F04C
:101C10002BF908BD62B608BDC0F8FF1FF0B589B04A
:101C200004460D461646FFF7DBFF5E2000F002F982
:101C30002B4B1A8801321A8072B6684629492A4607
:101C4000012300F071FB9DF8043084F82030029BE2
:101C500063629DF80C3084F8283008AB53F8135DAC
:101C600058689A68C4F82950C4F82D00C4F8312087
:101C70001B7B84F83530079BA363684600F0AAF904
:101C800062B604F11C05284600F0F8F9074650B981
:101C9000154C23685B682046144917229847204654
:101CA00003F06AFE19E0284600F0C2F90346E0633B
:101CB000B6FBF0F1284603FB116100F0A5F926649C
:101CC000094D2B685B682846094916229847284623
:101CD00003F052FE012384F84430384609B0F0BDC9
:101CE000C0F8FF1FE0F8FF1F78FDFF1FA8B200003B
:101CF000C0B20000006C70472DE9F041074690F833
:101D0000443013F0FF0F46D003F07CFC80460028DF
:101D100041D007F11C04204600F090F938B320466A
:101D200008F104014FF4807200F066F9002804DA2B
:101D3000BB6983B39847BDE8F0813B6C03443B64C7
:101D400000EBD07045107F2D0BD86E00C6F5807665
:101D500008EB450500231C46EA1894800233B34281
:101D6000FAD138464146002203F0C8FC10E0204674
:101D700000F078F9094B1B8823B1013B9BB2074A5D
:101D8000138013B95E2000F06FF8002387F8443009
:101D9000404603F093FCBDE8F08100BFC0F8FF1F90
:101DA000184B1A6842F480521A60174B174A1A608F
:101DB000174ADA6002F180421A61164A1A60164B1D
:101DC0001B7813F0010F07BF4FF41072134B4FF441
:101DD0000072134B1A60104B1B7813F0020F4FF474
:101DE00000720CBF0F4B104B1A600B4B1B7813F09B
:101DF000040F07BF4FF410720C4B4FF400720C4BE2
:101E00001A6070473C80044000C0024001401F003F
:101E10000110003800001F8074FDFF1F18B004403F
:101E200008C004401CB004400CC0044014B004407E
:101E300004C0044030B45E2810D84309084A012188
:101E400001FA03F514782C431470064A00F01F00C1
:101E5000814052F823400C4342F8234030BC704785
:101E6000DCF8FF1FC4F8FF1F5E2815D8430900F0F7
:101E70001F00012202FA00F0084A52F8231021EA5A
:101E8000000042F8230038B9054A012101FA03F3A2
:101E9000117821EA03031370704700BFC4F8FF1FD5
:101EA000DCF8FF1F10B582B002AB03F8011D026819
:101EB000546819460122A04702B010BD10B504466F
:101EC000C3691BB901230371002010BD00201871E4
:101ED000E06992B201F0D2FAE3691B7913B10123F0
:101EE0002371002010BD00BF00B583B0C06960B190
:101EF0000DF10701012200F0FBFF01280CBF9DF846
:101F000007004FF6FF7000B201E04FF0FF3003B062
:101F10005DF804FB30B583B00446C06978B10DF1BB
:101F20000701012200F0E4FF01280AD19DF80750C3
:101F3000E069C168013901F0C1F8284603E00020DA
:101F400001E04FF0FF3003B030BD00BF08B5C069FD
:101F500008B101F0EBF808BD2DE9F04104460E464A
:101F60009046002303714FF47A7282600373114B21
:101F70000360242007F06CFAE061B8B135460746EB
:101F800006F1200E3E4628686968AA68EB680FC60D
:101F9000103537467545F5D12868306004F10D00DD
:101FA00041460C2208F000FD002363762046BDE880
:101FB000F08100BFE0B20000002202714FF47A719C
:101FC0008160027302490160C2614273704700BFC1
:101FD000E0B20000014B0360704700BFE0B20000B8
:101FE0000D307047C3692BB19879012894BF002048
:101FF000012070470020704708B5C06910B100F09B
:1020000077FF08BD002008BD08B5C06928B101F000
:1020100055F8003018BF012008BD002008BD00BFE2
:10202000C3690BB1D86870474FF0FF30704700BFED
:10203000C3690BB1986970470020704738B50446F2
:10204000C36963B1FFF7F4FF05462046FFF7E8FFD9
:10205000281A47F6FF73984228BF184638BD00205B
:1020600038BD00BF10B50446C06930B101F08AF830
:10207000E06907F0F5F90023E36110BDC36923B1FE
:102080009879003018BF012070470020704700BFCA
:1020900010B58AB004460A4600238DF80830094975
:1020A00001918DF80A3001A82146012301F01CF9A5
:1020B000041C18BF012414B101A801F063F82046E4
:1020C0000AB010BD00B3000008B52AB101F0BAF99A
:1020D000003018BF012008BD012008BDF0B40C6815
:1020E000035D2F2B1CD101341AE0002563B11EE0E3
:1020F0000135013407F8013F0C2D05D016F8013FDA
:102100002F2B01D0002BF3D100235355035D2F2B30
:1021100008BF01340C60005D003018BF01200BE0E7
:102120000619035D2F2B08BF0025EDD0DDE7013434
:10213000137017460125E1E7F0BC70472DE9F04F19
:1021400099B082460F469146984600238DF81C3080
:10215000244A06928DF81E308DF840300F928DF88B
:10216000423001930C4606AE4FF0010B03E00FAC7A
:10217000234634461E46504601A902AAFFF7AEFF89
:10218000054680F00102204602A9D2B24346C84764
:1021900030B9BC421CD0204600F0F4FF00201EE005
:1021A0007DB13046214602AA5B4601F09DF8054606
:1021B000BC4211D0204600F0E5FF002DD8D1002010
:1021C0000DE0BC4206D0204600F0DCFF012006E016
:1021D000002004E0012002E00028C8D1002019B04E
:1021E000BDE8F08F00B3000038B504460A4601216F
:1021F00000F024FBB0B104F110052846214601226D
:1022000001F0EAFB28B928462146002201F0E4FB50
:1022100050B104F13800294600F040FE003018BFEC
:10222000012038BD002038BD002038BD2DE9F04F19
:1022300099B081469346019300238DF81C30394AAA
:1022400006928DF81E308DF840300F928DF8423096
:1022500006A8103100F022FE5C460FAE06AD4FF02E
:102260002F084FF0000A2CE023782F2B01D10134E6
:1022700027E03F1BFFB20C2F28BF0C2702A82146E6
:102280003A4608F091FB18AB3B4403F858AC304693
:1022900000F078FF3046294602AA012301F024F815
:1022A00040B9002389F804301E4AC9F8002089F893
:1022B000063032E03C44284600F064FF2B463546A9
:1022C0001E462046414608F0FFF807460028CBD1BD
:1022D000CBEB0404019B1C602B7989F80430114B73
:1022E000C9F800306B7989F80530AB7989F8063088
:1022F000AB68C9F80830EB68C9F80C302B69C9F82D
:1023000010302B7D89F81430AB69C9F81830EB69AF
:10231000C9F81C302B6AC9F82030484619B0BDE80E
:10232000F08F00BF00B30000F0B5A7B0044615461B
:102330001F4602A801ABFFF779FF01996E18695C8F
:1023400019BB9DF80C308DF85430344B14939DF824
:102350000D308DF855309DF80E308DF85630049BB9
:102360001693059B1793069B18939DF81C308DF8C8
:102370006430089B1A93099B1B930A9B1C9320466D
:1023800014A9274AFFF7E8FD45E000218DF8301039
:10239000224B0B938DF832109DF80E301BB920465E
:1023A000FFF70AFE37E00BA802A932463B4600F0D1
:1023B0009BFF18B92046FFF7FFFD2CE002A800F0B4
:1023C000E1FE17F0060F03D00BA8119900F076FE7E
:1023D0009DF830308DF87830104B1D939DF83130DA
:1023E0008DF879309DF832308DF87A300D9B1F933F
:1023F0000E9B20930F9B21939DF840308DF88830E1
:10240000119B2393129B2493139B259320461DA974
:102410003246FFF7A1FD204627B0F0BD00B3000013
:102420009CAE000008B500F1380308461946024A80
:102430000023FFF783FE08BD9120000008B500F1DE
:10244000380308461946024A0023FFF777FE08BD05
:10245000C9200000F0B59FB006460D46174649E07A
:102460009DF810401CB93046FFF7A6FD4BE0E52C67
:1024700040D02E2C3ED09DF81B1011F0080F39D102
:1024800000238DF83430214A0C928DF8363004A8A0
:10249000694600F0A3FC0CA8E9696A463B4600F0D7
:1024A00023FF18B39DF834308DF85830174B15932F
:1024B0009DF835308DF859309DF836308DF85A300A
:1024C0000E9B17930F9B1893109B19939DF8443004
:1024D0008DF86830129B1B93139B1C93149B1D93C8
:1024E000304615A96A46FFF737FD0CE03046FFF786
:1024F00063FD08E0E86904A900F098FD0028AFDC5E
:102500003046FFF759FD30461FB0F0BD00B3000064
:10251000084B00225A719A719A721A73022119613A
:1025200083F8302083F83C200349996383F83E20E8
:10253000704700BFE0F8FF1F00B30000084B1A68A7
:1025400042F480621A604FF00042DA62FF225A635E
:102550001A46D36A002BFCDA014B986BC0B2704765
:1025600000C0024010B50446164A174B1A6010F01E
:10257000010F02D0FFF7E2FF013C052C04D9032133
:1025800000231148114A02E06108F9D104E04263D6
:10259000023C01338B42FADB4CB10B4A0B48D36A45
:1025A00013F0F00FFBD05063936B023CF7D100297E
:1025B00007DD054AD36A13F0F00FFBD0936B0139A6
:1025C000F8D110BD00041F8000C00240FFFF009042
:1025D000064B1A6842F480621A604FF00042DA62D9
:1025E00058631A46D36A002BFCDA704700C00240D9
:1025F00008B505281ED8DFE800F003080D111519ED
:102600004FF038420E4B1A6017E04FF038420C4B37
:102610001A6012E00B4A0A4B1A600EE00A4A084B95
:102620001A600AE0094A064B1A6006E0084A044BA1
:102630001A6002E0074A024B1A60FFF7B1FB08BDBF
:1026400040F9FF1F000002B80000023801100138F5
:10265000010002380540013808B50079012102F077
:102660008DF8114B1B78F3B100220F4B1A700F4BF2
:102670001B78C3B113F0010F03D00D4B1A680D4B3B
:102680001A600A4B1B7813F0020F03D0084B5A68EC
:10269000094B1A60054B1B7813F0040F03D0044B51
:1026A0009A68064B1A6008BD44F9FF1FDCF8FF1F4B
:1026B000D0F8FF1F00E100E004E100E008E100E0E5
:1026C00010B5244B1B78002B3ED10122214B1A70F0
:1026D000214B1A68214B1B78002B28D072B61F4B58
:1026E0001B7813F0010F07D01D4B1C681D490968AA
:1026F00021401D4C21601960184B1B7813F0020F0C
:1027000007D01A4B1C68174949682140164C616074
:102710001960124B1B7813F0040F07D0144B1C6880
:10272000104989682140104CA160196062B6114BB4
:10273000DB68934208D00F4B0F491960DA6042F012
:1027400080421A610D4A1A600079002102F016F8E1
:1027500010BD00BF44F9FF1F40F9FF1FDCF8FF1F49
:1027600080E100E0C4F8FF1FD0F8FF1F84E100E023
:1027700088E100E000C0024001401F0000001F800F
:1027800038B5044683797BB1008940F20123984231
:1027900005D840F20225281AFFF7E4FE25812046DD
:1027A000FFF75AFF0023A37138BD00BF70B50E4676
:1027B000084B1C681D46A4B2FFF7C0FEFF2805D0D9
:1027C0002B689BB21B1BB342F6DB01E0012070BDFE
:1027D000002070BD50FCFF1FF8B505460F46164699
:1027E000FFF7CEFF2846FFF76BFF28464FF49671A0
:1027F000FFF7DCFF47F04000FFF7EAFE182426FA57
:1028000004F0C0B2FFF7E4FE083C14F1080FF6D163
:1028100027B1082F0CBF8720FF2000E09520FFF78D
:10282000D7FE0024FFF78AFEE87210F0800F03D075
:102830000134B4F5807FF5D1F8BD00BF2DE9F04F2C
:1028400083B0044601910023037383728371437143
:102850000271824B1F68BFB21046012101F08EFF4A
:102860002079012101F0BCFF2079012101F086FFD0
:102870007B4B1A6842F480521A600620FFF7B8FEBC
:10288000784B1A68784B1B78002B28D072B6764BA1
:102890001B7813F0010F07D0744B1868744909684E
:1028A00001407448016019606F4B1B7813F0020FF0
:1028B00007D0714B18686E49496801406D48416006
:1028C0001960694B1B7813F0040F07D06B4B186825
:1028D00067498968014067488160196062B6684B42
:1028E000DB68934200F0AB80654B66491960DA60A3
:1028F00042F080421A61644A1A60A0E02846FFF75D
:1029000067FE013E16F0FF06F8D1574B1B78C3B1A6
:1029100013F0010F03D0574B1A685C4B1A60524BEF
:102920001B7813F0020F03D0524B5A68584B1A60B1
:102930004D4B1B7813F0040F03D04E4B9A68554B48
:102940001A602046FFF7BCFE4FF00008DFF80C913C
:1029500009E0D9F80030DB1B9BB2B3F5FA6F02D95E
:102960000123637167E0204641464246FFF734FF8A
:102970000546E0720128ECD1204608214FF4D572BB
:10298000FFF72AFF10F0040F02D00123237310E099
:102990004FF00408FFF7D2FDE07208F1FF3313F0A7
:1029A000FF08F7D1AA2802D00223637143E0022373
:1029B0002373237B022B14BF4FF0000A4FF0804A91
:1029C0004FF037094FF00008DFF890B009E0DBF86E
:1029D0000030DB1B9BB2B3F5FA6F02D90823637199
:1029E00029E0204649464246FFF7F6FE20462921C7
:1029F0005246FFF7F1FEE0720028E8D1237B022B5C
:102A000011D120463A210022FFF7E6FE10B106233D
:102A1000637110E0FFF792FD00F0C000C02811D1F3
:102A2000032323730EE02046FFF716FE0198FFF7FD
:102A3000DFFD2E460DE02046FFF70EFE09E00A26D8
:102A4000FF255BE7FFF77AFDFFF778FDFFF776FDDF
:102A5000E9E7304603B0BDE8F08F00BF50FCFF1F30
:102A60003C80044040F9FF1FDCF8FF1F80E100E0DC
:102A7000C4F8FF1FD0F8FF1F84E100E088E100E008
:102A800000C0024001401F0000001F8000E100E084
:102A900004E100E008E100E070B504460E4B1D685B
:102AA0001E46ADB208E033689BB25B1BB3F5967F60
:102AB00002DD0F23637108E0FFF740FDE072FF289D
:102AC000F1D0FE2806D00D2363712046FFF7C4FD28
:102AD000002070BD012070BD50FCFF1FF8B50546F9
:102AE0000C4617461E46002B00F089801344B3F5B0
:102AF000007F7FDC83792BB103688B4202D103898D
:102B0000934216D92C602B7B032B18BF64022846F6
:102B100011212246FFF760FE10B103236B7169E0BB
:102B20002846FFF7B9FF002864D000232B8101233A
:102B3000AB713846FFF716FD3046334A334B1A6007
:102B400016F0010F07D0069A541CFFF7F7FC069BFE
:102B50001870701E0694052804D9032700232B49FA
:102B60002B4A02E04708F9D103E04A6301339F4250
:102B7000FBDCA0EB4700069A1044824219D21446AF
:102B80002249DFF88CC0CA6A12F0F00FFBD0C1F8FE
:102B900034C08B6BC3F30722227063700234A042EF
:102BA000F1D8069AD343034423F0010302331A44B5
:102BB000069200EB4700069B98420DD91C4613492C
:102BC000CA6A12F0F00FFBD08B6BC3F3072222709E
:102BD00063700234A042F3D82B8933449BB22B811B
:102BE000AA7A12B1B3F5007F0BD32846FFF7C8FDD0
:102BF0000120F8BD2846FFF72FFD0020F8BD012079
:102C0000F8BD0120F8BD00BF00041F8000C00240D5
:102C1000FFFF009000B583B0009200224FF40073D4
:102C2000FFF75CFF03B05DF804FB00BFF8B5064694
:102C3000214B186840F4806018604FF00040D86263
:102C40005963114602F500770446DA6A002A0FDB61
:102C5000FBE7DA6A002A14DBFBE7D36A002B1CDBF4
:102C6000FBE7112373713046FFF7F6FC0020F8BD37
:102C700008460A781D6845F480651D60DC625A6369
:102C8000E7E742781D6845F480651D60DC625A63A1
:102C90000231B942D9D1084ADFE7FF20FFF798FC9B
:102CA000FF20FFF795FCFFF749FCF07200F01F00D2
:102CB0000528D6D10120F8BD00C0024038B5044631
:102CC00015460B4611B9122343712BE0027B032AF0
:102CD00018BF4B0218211A46FFF77EFD10B10423DE
:102CE00063711FE02046FE212A46FFF79FFFC8B10F
:102CF00020464FF41671FFF759FD10B91523637183
:102D000010E020460D210022FFF766FD10B9FFF705
:102D100015FC10B11423637104E02046FFF79CFCFE
:102D2000012038BD2046FFF797FC002038BD00BFCA
:102D3000014A024B1A6070470000023840F9FF1F39
:102D400010B50446006A012104F1080200F0BAFD42
:102D5000034650B1E3693BB9A368E361637963F06B
:102D60007F036371012300E00123184610BD00BFFB
:102D700070B50646FFF7E4FF0346E0B1336AB26878
:102D8000023A197C02FA01F55A6915441C794CB1D2
:102D9000013D281900F0CCFC034660B1013C14F061
:102DA000FF04F6D1336A1B7C4FF400729A40B3697A
:102DB0001344B3610123184670BD00BF10B504462B
:102DC000006900F091FC20B1207D034B03EB401023
:102DD00010BD002010BD00BF54F9FF1F70B40023C8
:102DE0001A462E26C45C202C09D0DCB2082C02D155
:102DF000541C8E54E2B2541CC55C8D54E2B20133B3
:102E00000B2BEFD100238B5470BC70472DE9F001E0
:102E100000232022CA5401330B2BFBD1013800259B
:102E200007264FF008084FF00A0C1B4F21E02E2C0C
:102E300001D03A4606E00A2E24D04546664618E000
:102E4000A34221D012F8013F002BF9D1AE421DD38D
:102E5000A4F12103DBB25D2B1AD86B1CDBB20D444D
:102E6000A4F16102D2B2192A9CBF203CE4B22C70BA
:102E70001D4610F8014F002CD9D10878203818BF12
:102E8000012006E0002004E0002002E0002000E035
:102E90000020BDE8F001704707B3000038B50446D4
:102EA0000D4683790BBB91F82020102A07D102230D
:102EB00083710023C3614B8C5B0183610CE0202A8A
:102EC00014D103238371496AC161284604F11802B1
:102ED00000F084FC034648B125620123637100229F
:102EE000A260E2602261227500E00023184638BD2E
:102EF0002DE9F04F85B00446884603928379002B74
:102F000069D0437913F0010F68D08269C368D11A80
:102F10000398884201D98BB20393039B002B57D0AF
:102F20001E46DFF8FCA0DFF8FC90DFF8FCB0E36899
:102F3000C3F30807A279022A04D1226A516A01EB7D
:102F400053211BE0206A0579013D05EA5325EDB2C6
:102F50005FB955B913B9E369A36006E0224652F898
:102F6000081F00F005FC00283BD0226AA368023B42
:102F7000117C03FA01F1526911442944C7F5007329
:102F80009E42C6BF1D46ADB23546637913F0400F71
:102F900002D1B5F5007F39D1D9F8003099422AD154
:102FA00034E0A8440DE057447819874209D03B46E5
:102FB000424613F8011B02F8011B8342F9D1C71BDB
:102FC000B844E3682B44E360761BB6B2002EAED162
:102FD000039B98B20DE04FF6FF700AE04FF6FF70CA
:102FE00007E04FF6FF7004E04FF6FF7001E04FF688
:102FF000FF7000B211E0CDF80080DBF800003A4627
:103000002B46FFF76BFD0028CBD1EDE708460021EA
:1030100000F06AFB0028C6D1E9E705B0BDE8F08FF3
:1030200054F9FF1F988FFF1F50F9FF1F70B5054619
:103030000C468379012B1CD9C36813F01F0F1AD1DA
:10304000202609E0237883B1E52B05D02E2B03D071
:10305000E37A13F0080F10D0284621463246FFF7D6
:1030600047FFC0B243B2202BECD040F3C011C8B22E
:1030700004E0FF2002E0FF2000E0202040B270BD0D
:1030800030B583B004468379012B0FD9C5680DF1A3
:1030900007010122FFF72CFF012809D1E3681F3344
:1030A000E36005F4F070044B184402E0002000E0F7
:1030B000002003B030BD00BF54F9FF1FF8B504462F
:1030C0000F4683797BB382698A422BD3022B02D1CC
:1030D000E160012327E021B900238360C36001235D
:1030E00021E0C368026A157C09355A1EEA4001399D
:1030F00021FA05F5AA4200D813B9E369A3600AE0F2
:10310000AD1A08E0206AA168324600F031FB013DAB
:10311000034610B907E004F10806002DF2D1E7607C
:10312000012300E000231846F8BD00BF38B504466F
:10313000807918B394F90530002B1BDA2046012161
:10314000FFF73CFE0546C0B1A379012B9CBFA369E4
:10315000C361A38B4383E38B8382094B1B682BB131
:10316000183005F1160198472B8B6B82637903F0B9
:103170007F03637100F08CFA38BD002038BD00BFBA
:1031800048F9FF1F10B50446FFF7D0FF034610B102
:103190000023A3710123184610BD00BFF0B583B012
:1031A00004460D468379012B4ED1427902F002028A
:1031B00002F0FF01002A49D08269AA4248D3002ABE
:1031C00047D0C6682946FFF779FF0346002840D05C
:1031D0004DB9206AE16900F0D9FB0346002838D0D8
:1031E0000023E3611DE0206AA16801AA00F0C0FA93
:1031F000A8B1206A019990F820704FF6F872164B2A
:10320000102F08BF134699420BD200F0BFFB30B11C
:10321000206AA1686FF0704200F00CFB08B900232F
:1032200017E0A561637963F07F0363712046FFF7C0
:103230007DFF034668B12046B54234BF294631467A
:10324000FFF73CFF034604E0002302E00B4600E0EA
:103250000023184603B0F0BDF8FFFF0F38B5044651
:1032600015461F4B03EB4113DA7A12F0110F02D00F
:1032700015F0420F2CD121751A4A12682261998AE1
:103280000904E1615A8B1143E161D87A10F018000A
:1032900004D1DB69A3610123A3710AE0102819D1CD
:1032A000206A04F1180200F099FA0346A8B1042339
:1032B000A37105F00F0363710023A360E36015F0B1
:1032C000400F09D020461946FFF768FF034604E087
:1032D000002302E0002300E00123184638BD00BFB0
:1032E00054F9FF1F988FFF1F2DE9F04F85B0054659
:1032F0000C469A468679002E7FD1104601A9FFF729
:1033000085FD00287BD0236A2B620027A760E76039
:10331000DFF8FC904FF0010825E0C1F3431B204685
:10332000FFF7AEFE014600286AD003780BB1E52B0B
:1033300009D12FB985F814B0D9F800302B61474670
:103340000B7883B913E001A80B2206F02DFB50B9CE
:103350000AF03003302B53D0284659465246FFF727
:103360007DFF06464CE0E168A3699942D5D30AF097
:103370001203122B44D137B128460121FFF71EFD5D
:10338000044660B93CE0A379022B39D02046FFF710
:10339000EFFC0646002833D000232B751A4C20463C
:1033A0000021202206F094FB01AB03CB206061607A
:1033B0001A889B782281A372144B1B682BB104F1ED
:1033C000100004F10E01984707E0212323742823FD
:1033D00063740023A3730823E373238A6382238324
:1033E000E389E38200F054F9064648B12846297D76
:1033F0005246FFF733FF064602E0002600E006468D
:10340000304605B0BDE8F08F54F9FF1F48F9FF1FA3
:10341000988FFF1F10B504460021FFF7BFFE03463B
:1034200068B120460121FFF7C9FC38B1E5220270DE
:103430000023A37100F02CF9034600E00023184696
:1034400010BD00BF10B58AB004460A4600238DF8AF
:103450000830094901918DF80A3001A8214602235C
:10346000FFF742FF034618B101A8FFF7D3FF034659
:1034700018460AB010BD00BF00B300002DE9F04FA0
:1034800085B00446884601928379012B40F0BE80C6
:10349000437913F0020F00F0B98013F0040F08D045
:1034A0008169C3688B4204D0FFF708FE002800F052
:1034B000AD80019A002A00F08C801646DFF8B0A19A
:1034C000DFF8B0B1206AE76890F8049009F1FF399D
:1034D00009EA5729C7F3080719F0FF0929D1002F76
:1034E00040F0AA80A16851B9E36933B92046FFF7DB
:1034F00027FC002840F08E8088E0A3608AE003AAC1
:1035000000F036F9002800F0A880039B226A92F8A8
:1035100020004FF6F871524A102808BF0A4693421D
:1035200005D32046FFF70CFC002873D16EE0A360A2
:1035300070E0C7F50075ADB2AE4238BF3546A3683E
:10354000023B027C9340426913449944B5F5007FE5
:1035500012D1DBF800304B4504BF4FF0FF33CBF8FE
:103560000030404B186849464246FFF7A7FB002849
:103570004CD008F5007824E07FB9E268A3699A424C
:103580000BD300F085F8002840D0CBF80090364AE5
:10359000137843F00103137005E04846012100F061
:1035A000A3F8002832D057447819874209D03B4607
:1035B000424612F8011B03F8011B8342F9D1C71BD5
:1035C000B844761BB6B2E3681D44E560002E7FF474
:1035D00079AFE368A269934205D9A361637963F087
:1035E0007F03637108E0214B1B682BB1019B1BB16A
:1035F000637963F07F036371637913F0080F03D07D
:103600002046FFF793FD08B1019826E001232371BE
:10361000002022E0B6F5007F34BF35464FF4007538
:10362000236AA268023A197C02FA01F95B6999449B
:10363000B5F5007FA1D18CE7C7F50075ADB2AE42FC
:1036400038BF3546A368023B027C03FA02F943699E
:103650009944B5F5007FA0D17BE705B0BDE8F08FB8
:10366000F8FFFF0F50F9FF1F54FBFF1F48F9FF1F22
:1036700054F9FF1F988FFF1F00B583B002AB03F80A
:10368000011D19460122FFF7F9FE03B05DF804FBA6
:1036900008B5104B1B78D3B10F4B18680F4B196846
:1036A0000F4AFFF70BFB034690B10E4B196849B167
:1036B000094B18680A4AFFF701FB034640B1002294
:1036C000084B1A600022034B1A70012300E001230B
:1036D000184608BD54FBFF1F50F9FF1F988FFF1FAE
:1036E00054F9FF1F4CF9FF1F38B504460D460C4B2B
:1036F0001B6883420DD0FFF7CBFF034670B1094B27
:1037000018682146084AFFF785FA034630B1044B92
:103710001C60064B1A7815431D700123184638BDEE
:10372000988FFF1F50F9FF1F54F9FF1F54FBFF1F15
:1037300010B50446FFF7ACFF034680B109494B1EA4
:1037400001F2FF11002203F8012F8B42FBD1064B3F
:103750001C60064B1A7842F001021A7001231846C9
:1037600010BD00BF54F9FF1F988FFF1F54FBFF1FB0
:1037700070B504460D461646C36801338B4225D307
:10378000C36990F82020102A0CBF080AC809184401
:10379000104B1B68984204D00021FFF7A5FF034699
:1037A000A8B194F82030102B06D1EDB20A4B33F8B3
:1037B0001530336001230AE005F07F05064B53F80E
:1037C000253023F070433360012300E000231846C6
:1037D00070BD00BF988FFF1F54F9FF1F2DE9F04304
:1037E00083B0044602AE46F8041D914600254FF40E
:1037F00000780F4F204601993246FFF7B9FF034684
:1038000088B1237C08FA03F31D4494F820104FF686
:10381000F873102914BF39461946019B8B42E9D32E
:10382000C9F800500123184603B0BDE8F08300BF7B
:10383000F8FFFF0FF8B504460D461746012931D9A8
:10384000C368013399422FD8C36990F82020102A09
:103850000CBF0E0ACE091E44164B1B689E4205D0B3
:1038600030460021FFF740FF034600B394F82030B4
:10387000102B04D1EDB2104B23F8157004E005F0C5
:103880007F050D4B43F825700C4B1A7842F001026E
:103890001A70237E012B09D9A3681E44084B1E60B1
:1038A000012304E0002302E0002300E00123184686
:1038B000F8BD00BF988FFF1F54F9FF1F54FBFF1F77
:1038C0004CF9FF1F2DE9F04F85B006468A4600925D
:1038D00017681FB101370023019305E0076801292C
:1038E00014BF002301230193F36803F10108DBB146
:1038F0003C4600254FF00209CB46A0453CBF4C4654
:103900005F463046214603AAFFF732FF60B1039BB2
:103910000BB1671C03E0631CDB1B534506D001356C
:103920000134F368AB42E8D800232AE03046214650
:103930006FF07042FFF77EFF034648B921E0651E35
:10394000304629462246FFF775FF034618B918E0AE
:10395000BC42F4D803E0BD4201D92C46EFE7009BFE
:10396000196829B130463A46FFF764FF034640B173
:10397000009B1F60019B1BB101373760012300E0F2
:103980000123184605B0BDE8F08F00BFF0B583B045
:1039900005460C460223036000260E4F28462146AA
:1039A00001AAFFF7E5FE80B1284621463246FFF71F
:1039B00041FF50B1019C95F820104FF6F873102983
:1039C00018BF3B469C42E9D301E0002000E0012003
:1039D00003B0F0BDF8FFFF0FF8B50546494B19607D
:1039E0001446DAB1042A7FD800200146FFF77CFE96
:1039F0000346002800F08380434B03EB041494F843
:103A0000AE3104F5D47413F07F036FD1D4F81210E3
:103A1000632974D9D4F80E400CB970E00024204614
:103A20000021FFF761FE0346002868D0364BB3F84B
:103A30000B30B3F5007F5BD1334B1B7C002B5ED08A
:103A4000314AD289002A55D02F4A517B002953D0C0
:103A50002B76297100232B74012003E05A1C2A7451
:103A6000072B4BD82B7C1E4600FA03F29142F5D16E
:103A7000254BD98A01B9596AA960234BDA892244B6
:103A8000EA61B3F8110087B268841B7C03FB012351
:103A90006B627A0102F2FF1203EB62236B611A4A36
:103AA000B2F813200AB9184A126AE31A134423FA27
:103AB00006F6EE6040F6F4739E4204D80C2385F8B7
:103AC000203001231BE04FF6F4739E4204D81023EC
:103AD00085F82030012312E00B4BDB6A6B62202358
:103AE00085F8203001230AE0002308E0002306E0E7
:103AF000002304E0002302E00B4600E00023184608
:103B0000F8BD00BF50F9FF1F54F9FF1F0B4B1B7886
:103B100013B90B4B1B7873B10A4B1B78202B03D9BD
:103B20000123037100207047581C064A1070064A92
:103B3000D154012070470020704700BFBEFBFF1F1B
:103B400080FBFF1FBFFBFF1F5CFBFF1F704700BF19
:103B5000024B1878024B1B78C01A7047BDFBFF1F41
:103B6000BCFBFF1F074B1B78074A12789A4205D906
:103B7000591C044A1170054AD05C70474FF0FF3061
:103B8000704700BFBCFBFF1FBDFBFF1F84FBFF1F77
:103B9000054B1B78054A12789A4286BF044AD05CCE
:103BA0004FF0FF30704700BFBCFBFF1FBDFBFF1F86
:103BB00084FBFF1F08B5104BDB7813F0200F0CD1EE
:103BC000122000F0B3FD0D4B1B689BB100210C4A85
:103BD00011700C4A1078984708BD0B4A13780133CE
:103BE000DBB21370012B02D8084B1B7813B91220DB
:103BF00000F09CFD08BD00BF0060064058FBFF1FA1
:103C0000BCFBFF1FBDFBFF1FA8FBFF1F80FBFF1FAF
:103C100038B514460D4B1B7813B90D4B1B7893B177
:103C20000C4B1D78C5F12103A34202D2012202717F
:103C30001C4609482844224600F0B4F82544054BA8
:103C40001D70204638BD002038BD00BFBEFBFF1FE1
:103C500080FBFF1FBFFBFF1F5CFBFF1F00220271E9
:103C60004FF47A7181600273014A0260704700BFAD
:103C700020B3000008B53D4BDB78DBB213F0100F2A
:103C800006D01021394AD17013F0400F03D108BD7E
:103C900013F0400F2CD013F0040F1BD00023344A34
:103CA0001370344A1370344B1B681BB19847314B67
:103CB0001B782BB901222F4B1A7000222F4B1A7040
:103CC0002A4BD0229A702D4A12781A7101222C4B5D
:103CD0001A7009E00122264B1A700022294B1A7033
:103CE000224BC0229A701B790222204BDA7008BD49
:103CF0001E4A927812F0100F1CD013F0010F14D14D
:103D00001F4B1B781B4A12789A4207D9591C1C4A30
:103D100011701A4AD25C154B1A7102E00022134B43
:103D20001A71D022114B9A701BE0104BC0229A706E
:103D30001B7916E00022144B1A701220134903223B
:103D400000F0ACFC094B1B79DAB20E4B1B781F2B31
:103D500007D80749097821B1581C0A4908700C494D
:103D6000CA540222014BDA7008BD00BF0060064051
:103D700055FBFF1FBFFBFF1FA4FBFF1F5CFBFF1FCB
:103D8000C0FBFF1FBDFBFF1FA8FBFF1FB53B0000D3
:103D900084FBFF1F08B50248FFF760FF08BD00BFA6
:103DA000ACFBFF1F844641EA000313F003036DD10F
:103DB000403A41D351F8043B40F8043B51F8043BEE
:103DC00040F8043B51F8043B40F8043B51F8043BF5
:103DD00040F8043B51F8043B40F8043B51F8043BE5
:103DE00040F8043B51F8043B40F8043B51F8043BD5
:103DF00040F8043B51F8043B40F8043B51F8043BC5
:103E000040F8043B51F8043B40F8043B51F8043BB4
:103E100040F8043B51F8043B40F8043B51F8043BA4
:103E200040F8043B51F8043B40F8043B51F8043B94
:103E300040F8043B403ABDD2303211D351F8043B34
:103E400040F8043B51F8043B40F8043B51F8043B74
:103E500040F8043B51F8043B40F8043B103AEDD2E3
:103E60000C3205D351F8043B40F8043B043AF9D234
:103E7000043208D0D2071CBF11F8013B00F8013B07
:103E800001D30B8803806046704700BF082A13D314
:103E90008B078DD010F003038AD0C3F10403D21A2C
:103EA000DB071CBF11F8013B00F8013B80D331F860
:103EB000023B20F8023B7BE7043AD9D3013A11F8E0
:103EC000013B00F8013BF9D20B7803704B7843704B
:103ED0008B7883706046704730B4394A394913682B
:103EE00013F0800FFBD10B6813F0800FF7D172B67F
:103EF000354B1B78002B5FD0344B1C6804331D6896
:103F0000043318680433196804331A6804331B68CF
:103F10002C44204401440A441A44C2F34E0242F4A1
:103F200000422B4B1A602C331C6804331D68043389
:103F300018680433196804331A6804331B682C4466
:103F4000204401440A441A44C2F34E0242F400429F
:103F5000204B1A6003F108131C6804331D680433F6
:103F600018680433196804331A6804331B682C4436
:103F7000204401440A441A44C2F34E0242F400426F
:103F8000154B1A602C331C6804331D680433186801
:103F90000433196804331A6804331B682C44204422
:103FA00001440A441A44C2F34E0242F400420B4B4D
:103FB0001A600022044B1A7062B630BC704700BF12
:103FC00024B0034024B00B40C2FBFF1F38B00340B5
:103FD0002CB0034030B003402CB00B4030B00B404D
:103FE00060223A4B1A70E12201331A70384B1B7869
:103FF000082B10D1012203F1804303F56C331A60C2
:10400000132334490B6001F5FF2101F2FC710A60B2
:10401000314A13601FE00A2B0DD119222F4B1A6071
:1040200013232C490B6001F5FF2101F2FC710A609A
:10403000294A13600FE00C2B0CBF15223D22274BA1
:104040001A60122323490B6001F5FF2101F2FC7174
:104050000A60214A1360224B1B7833B10123214AA5
:10406000136002F50022136005E000231D4A13606F
:1040700002F5002213601C4B1B78012B06D880230D
:104080001A4A136002F5002213601AE0042B06D8C6
:104090008423164A136002F50022136011E0082BF6
:1040A00006D88523114A136002F50022136008E048
:1040B000102B94BF862387230C4A136002F500223D
:1040C000136001220A4B1A70704700BF004007407E
:1040D0009C8FFF1F0CB003400CB00B4008B0034096
:1040E000C5FBFF1F20B003409D8FFF1F24B003407E
:1040F000C2FBFF1F2DE9F8430D2813D9172802D85A
:104100000E38C0B20EE0A0F11A03DBB2052B02D8C4
:104110000938C0B206E0A0F12203DBB2062B73D847
:104120001838C0B23A4B1E5C3A4B1B780BB1FFF704
:10413000D3FE16F0800F29D172B6374C374D4FF0B1
:10414000010726602F7062B672B6236813F0800FE5
:1041500004D12B7813F0FF0F0FD1F2E7304B186822
:1041600000222E4B1A7062B62E4B1B781841BDE808
:10417000F8832B7813F0FF0FE3D062B601F006FE50
:1041800072B6236813F0800FF3D0E7E772B606F03B
:1041900040095FFA89F9244F244C06F03F06244D6C
:1041A0004FF00108B9F1000F04D03B6823F0100371
:1041B0003B6003E03B6843F010033B60266085F8FA
:1041C000008062B672B6236813F0800F04D12B789A
:1041D00013F0FF0F0FD1E5E7164B18680022144BC0
:1041E0001A7062B60F4B1B781841BDE8F8832B7824
:1041F00013F0FF0FD6D062B601F0C8FD72B6236887
:1042000013F0800FF3D0E7E70020BDE8F88300BF8C
:1042100038B30000C2FBFF1F00B00340C4FBFF1F08
:1042200010B00340C1FBFF1F0CB00B4000B00B40AF
:10423000C3FBFF1F10B00B40024A137813F0010FAD
:10424000FBD070470100024010B584B0174B6C469C
:10425000186859689A68DB680FC4154B1B7813F00F
:10426000020F19D08022134B1A70332204331A70B4
:104270000322013B1A7072B66B4643F001030E4CE9
:104280002046984762B6237813F0700304D0237059
:1042900009E0013B03D106E044F6216304490A78B2
:1042A00012F0010FF5D004B010BD00BF50B30000F4
:1042B00001000240070002400000024010B5044621
:1042C000B0F5006F0AD2064B1B7813F0010F01D135
:1042D000FFF7BAFF04F1A054207810BD002010BDF4
:1042E0000100024038B504460D46B0F5006F0ED20D
:1042F000074B1B7813F0010F01D1FFF7A5FF04F165
:10430000A0542378AB4202D02570FFF795FF38BD4B
:1043100001000240024B1A6801321A60704700BF68
:1043200050FCFF1F08B50D4C236813F4802F01D0FB
:1043300000F0F0FB236813F4806F01D001F0F2FF6E
:10434000236813F4006F01D002F0EAFA236813F433
:10435000805FE9D002F074FDE6E700BF34800440DE
:1043600008B5FFF7DFFF00BF1022014B1A8070472E
:1043700000200540704700BF024A136818441060CF
:1043800018467047A08FFF1FFEE700BFEFF31383AF
:10439000ABB9EFF31083ABB9EFF3058323B10F2B68
:1043A00005D9094A985C03E04FF4807000E00020D2
:1043B000EFF311833BB1834238BF184670474FF08B
:1043C000FF30704700207047F0E300E010B5154B58
:1043D0001C681C6014F4805F05D0134BDB6813B1BC
:1043E000114BDB68984714F4005F05D00E4B1B6936
:1043F00013B10D4B1B69984714F0200F05D00A4BE1
:104400001B6E13B1084B1B6E984714F0100F07D0AA
:10441000054BD3F884301BB1034BD3F88430984755
:1044200010BD00BFA0900440C8FBFF1F10B5274B74
:104430001C681C6014F4803F05D0254B1B6813B129
:10444000234B1B68984714F4003F05D0204B5B6852
:1044500013B11F4B5B68984714F0010F05D01C4B3C
:104460001B6C13B11A4B1B6C984714F0020F05D04C
:10447000174B5B6C13B1164B5B6C984714F0080F2D
:1044800005D0134B9B6C13B1114B9B6C984714F0E8
:10449000040F05D00E4BDB6C13B10D4BDB6C984752
:1044A00014F4002F05D00A4B5B6E13B1084B5B6E02
:1044B000984714F4802F07D0054BD3F880301BB1F8
:1044C000034BD3F88030984710BD00BFA0A0044034
:1044D000C8FBFF1F10B5384B1C681C6014F0080F98
:1044E00005D0364B5B6A13B1344B5B6A984714F0C6
:1044F000100F05D0314B9B6A13B1304B9B6A984724
:1045000014F0400F05D02D4BDB6A13B12B4BDB6A47
:10451000984714F0800F05D0284B1B6B13B1274B25
:104520001B6B984714F0200F05D0244B5B6B13B125
:10453000224B5B6B984714F0010F05D01F4BDB6BD0
:1045400013B11E4BDB6B984714F0020F05D01B4BC9
:104550009B6D13B1194B9B6D984714F0040F05D058
:10456000164BDB6D13B1154BDB6D984714F4007FD0
:1045700005D0124BDB6E13B1104BDB6E984714F471
:10458000807F05D00D4B1B6F13B10C4B1B6F9847F1
:1045900014F4806F05D0094B5B6F13B1074B5B6F51
:1045A000984714F4006F05D0044B9B6F13B1034B75
:1045B0009B6F984710BD00BFA0B00440C8FBFF1F11
:1045C00010B5264B1C681C6014F0010F05D0244B5D
:1045D0009B6813B1224B9B68984714F0800F05D05D
:1045E0001F4B5B6913B11E4B5B69984714F0100FAA
:1045F00005D01B4B9B6913B1194B9B69984714F06D
:10460000040F05D0164BDB6913B1154BDB699847D6
:1046100014F0080F05D0124B1B6A13B1104B1B6A24
:10462000984714F0020F05D00D4B9B6B13B10C4B48
:104630009B6B984714F0200F05D0094B1B6D13B1ED
:10464000074B1B6D984714F0400F05D0044B5B6D72
:1046500013B1034B5B6D984710BD00BFA0C0044071
:10466000C8FBFF1F10B50B4B1C681C6014F0020F39
:1046700005D0094B9B6E13B1074B9B6E984714F006
:10468000010F05D0044BDB6F13B1034BDB6F984771
:1046900010BD00BFA0D00440C8FBFF1F30B42128CC
:1046A00031D8042A2FD8DFE802F00709050B0300F0
:1046B0000B2406E00A2404E0082402E00C2400E0B5
:1046C0000924124B03EBC0035A68114B114DC3F878
:1046D0009C51114DC3F8A051104DC3F8A451104D79
:1046E000C3F8A8510F4DC3F8AC5172B6136823F448
:1046F000702313600C4D45F8201043F0807343EA9B
:104700000444146062B630BC704700BF60B3000060
:10471000008AFF1FCD4300002D440000D544000057
:10472000C145000065460000C8FBFF1F094B03EBB5
:10473000C0035A6872B6136823F0877323F480337A
:1047400043F0807313600022034B43F8202062B6CD
:10475000704700BF60B30000C8FBFF1F044B00227E
:104760001A6004490A60044A106010221A607047F7
:1047700014D0034004D0034000D0034021281ED8A9
:104780000F4B53F8303093F8802212F0FF0F08D00F
:1047900019B1012283F880207047012283F800219B
:1047A0007047074B03EBC000436821B11A6842F021
:1047B00003021A6070471A6822F002021A607047FA
:1047C00060B30000212806D8044B53F8303093F82A
:1047D0000002C0B270470020704700BF60B3000005
:1047E00021281CD80E4B03EBC0035B68012908D1BC
:1047F0000B4A52F8302082F880124FF4A2721A60ED
:104800007047074A52F83020002082F8800219B918
:104810004FF480721A60704740F203121A607047BA
:1048200060B3000072B60D4B1B680D4A12680D494B
:10483000096862B611F0806F02D0322B88BF013256
:10484000C3F58C3303F23F130749A1FB03031B0994
:104850004FF47A7000FB0230704700BF18E000E0B0
:1048600050FCFF1F04ED00E0398EE33838B50546F3
:10487000FFF7D8FF044625B938BD013D0AD004F53D
:104880007A74FFF7CFFF001BB0F57A7FF5D201F005
:104890007DFAF6E738BD00BF10B5254B4FF4000296
:1048A0001A604FF080721A604FF000721A604FF079
:1048B00080621A604FF000621A6000201D4B186081
:1048C00048F6FF710433196028231B4A136008322D
:1048D0001360083213600832136008321360083224
:1048E000136008321360083213600922134C2260EF
:1048F00004F58054043420600434216004342360BF
:1049000008342360143C226004F5FE240434206043
:104910000B4801600B490B6008310B600A4B1A60B1
:10492000FFF75EFBFA20FFF7A1FF00F073FC10BD5C
:1049300008E100E0048003400C8003400080034055
:1049400008800B400C800B4000800B4030B40E4BB5
:104950001B7843F002020D4C04EBC20460600C486B
:10496000007800280CBF8824C82444EA0141074D80
:1049700045F8321080F00100054A107083F0010301
:10498000014A137030BC7047BCFCFF1F0080FF1F42
:1049900035FDFF1F10B4431E032B11D872B60A4A0F
:1049A00052F8230050B14268074941F82320074AD2
:1049B00032F813400188611A22F8131062B600E041
:1049C00000205DF8044B7047ACFCFF1F7CFFFF1F0D
:1049D000013803280DD872B6074B53F820302BB19D
:1049E000002001305B68002BFBD100E0002062B6A4
:1049F00070470020704700BF00FDFF1F38B572B63A
:104A000001231B491B4C5A1812F8012C12F0080FF5
:104A100024D09A0054F832506DB9164B03EBC20102
:104A200008304860144943F83210144B1A78013AA0
:104A30001A7062B638BD42F0010254F832506DB9B6
:104A40000C4B03EBC201083048600D4943F83210AB
:104A50000A4B1A78013A1A7062B638BD0133052B39
:104A6000D1D162B60022054B1A7000F037FC38BD78
:104A700098B400000080FF1F880040002AFDFF1F3F
:104A8000C800400010B4431E032B37D8400140F04B
:104A900010001C4A104472B61B4AD25C032A09D883
:104AA000DFE802F019021B050830022216E0083088
:104AB000042213E0154A52F823201AB9134A42F887
:104AC000231003E0124A52F823205160104A42F8A2
:104AD000231062B612E0032200E005220A4CE254E1
:104AE00001F10803436000F00803002B0CBF88238A
:104AF000C8230A8843EA0243036062B65DF8044BA8
:104B0000704700BF0080FF1F68FCFF1F00FDFF1FF4
:104B100010FDFF1F2DE9F84FA34CDFF8E092DFF8FE
:104B2000E0A2DFF8E0B22578EDB215F0040F1DD059
:104B30009E4B1B7813F0FF0F16D09D4B1B7803F094
:104B4000FF022BB1531EDBB2994A137003B900BEAA
:104B5000984B1B7803F0FF0233B1531EDBB2954A2A
:104B600013700BB900F0FAFC0423237015F0080F42
:104B700000F0E48299F80030DBB21D0940F0218298
:104B80008D4D9E0805EBC6035A6855F83630C3F3C1
:104B90008303013B0C2B00F21082DFE813F0CB0102
:104BA000CB010E020E020E020E020E020E02E801F0
:104BB0000E020E020E020D00804913680B6052684F
:104BC0004A607F4A45F8362000227E490A607A49C9
:104BD0000A618A6101217C4A11709BB240F28162B4
:104BE000934218D8B3F5D06F2ED2B3F5817F00F081
:104BF0001E8106D8802B00F0C980822B00F0CC806B
:104C000066E140F20232934200F02681B3F5A06FD4
:104C100000F062815CE142F22102934200F0868161
:104C200007D8B3F5086F00F0AB80B3F5106F11D063
:104C30004EE142F22122934200F0418142F22132C0
:104C4000934200F0498143E1604B5D68002D40F0E4
:104C5000188130E1594B9A78544B1A70564D05F132
:104C600080062B6A13F0800F03D0686A083800F0C2
:104C700035FB0835B542F4D1DFF88C810026374684
:104C8000534AB05828B1456800F028FB0DB12846BA
:104C9000F9E700234E4973504E4AB3504E4BF0583B
:104CA00028B1456800F01AFB0DB12846F9E700234A
:104CB00049497350494AB35028F8023F484BFB5CBE
:104CC000023B032B0AD8DFE803F0020602060022AB
:104CD000434BDA5502E00122414BDA5501370436E5
:104CE000102ECDD100223F4B1A7001253E4EDFF829
:104CF0001C81314F05EB080313F8013C06F8043B17
:104D000013F0080F2DD000F0C9FA48B1A90007EB45
:104D1000451200F108035360344A47F8312007E098
:104D2000AB00002247F833202E4B1A7801321A705C
:104D300000F0B4FA58B1AB0043F0010307EBC30134
:104D400000F108024A601E4A47F8332009E0AB0030
:104D500043F00103002247F83320224B1A78013236
:104D60001A70AA0042F00201002347F8313042F0E5
:104D7000030247F8323001351D4B9E42BAD11EE284
:104D80000A4B1B781B4D2B700127AAE0194D0023FD
:104D90002B706B700227A4E0084B9B88042B37D93B
:104DA0000F22154B1A70C1E08020074034FDFF1F11
:104DB000BDFCFF1F36FDFF1F0080FF1F20FDFF1FF2
:104DC000C800400054FCFF1F35FDFF1F9CB40000CD
:104DD000ACFCFF1F58FCFF1F00FDFF1F10FDFF1F55
:104DE00068FCFF1F2AFDFF1FC42007408800400009
:104DF000D42007402CFDFF1FC02007409020074013
:104E000094200740982007407AFFFF1F98B40000C5
:104E1000A04A0021117051709F4A12F8233013F0FC
:104E2000020F5CD09B4D01232B70022759E09B4B56
:104E30009B8803F07F03042B02DC984A52881AB146
:104E40000F22954B1A7071E0934A12F8231021F04B
:104E5000020102F82310B2E1904B9B8803F07F031C
:104E6000042B02DC8D4A52881AB10F228A4B1A7029
:104E70005CE0894A12F8231041F0020102F8231085
:104E80009DE1864B5E889F88854BA3F10C021146FD
:104E900033F80C0CB04209D133F80A0CB84205D1F2
:104EA000360A032E0CBF2F7817891AE00D690C33D0
:104EB0000C32002DEBD10F22774B1A7036E0794B74
:104EC0001A68794B1A60754B9A78784B1A7076E1AC
:104ED0000F22714B1A7029E000273D4601E002279E
:104EE0006C4D6E4BDB889F4228BF1F46402F34BF5E
:104EF0003E46402628463146FFF728FD3544BF1B75
:104F000003D13F2E00F2608110E0402F34BF3E46B7
:104F1000402628463146FFF719FD3544BF1B01D115
:104F20003F2E03D9624B1D60624B1F8001238AF81C
:104F3000003042E0594B198842F22103994212D1C4
:104F40005D4BD81D12F8011B03F8011F8342F9D1F4
:104F50005A4B1B68862B02D10F22594B1A70002026
:104F60000146FFF7F3FC574B45F8363025E0504B30
:104F70001E68BEB14F4FB7F80080B8F1400F34BF84
:104F80004546402530462946FFF7E0FCC5EB0803BF
:104F90009BB23B800BB9402D01D1354400E0002588
:104FA000434B1D603D4B1B88B3F5A06F05D13B4BB8
:104FB00000225A709B788BF8003001238AF8003069
:104FC000B9E0414E9F0806EBC708D8F80420A2F1CB
:104FD0000800013DEDB213F0080F47D000F07EF954
:104FE0003A4B53F825304BB35A68384941F82520DD
:104FF00003F10802C8F80420354A525D032A12D88A
:10500000DFE802F002060A0E0321314A51550AE098
:1050100002212F4A515506E005212D4A515502E043
:1050200004212B4A515518F0080F0CBF8822C822C2
:105030001B8842EA034346F837307CE0244B5B5D33
:10504000032B0BD8DFE803F0777702060022204B12
:105050005A5570E001221E4B5A556CE018F0080FAB
:105060000CBF022203221A4B5A5564E056F837301F
:105070001B0C22F8083C002B55D0002322F8063CDC
:1050800042F8043C134B53F825302BBB114B43F82B
:10509000250025E02CFDFF1FC020074020FDFF1F3D
:1050A000A8B4000050FCFF1F8CFFFF1F44FDFF1F32
:1050B00054FCFF1F28FDFF1F83FFFF1F84FFFF1FFE
:1050C000BDFCFF1FC80040000080FF1F00FDFF1F48
:1050D00068FCFF1FACFCFF1F3F4B53F825305860A6
:1050E0003D4B43F825003D4B33F8151032F8082CA2
:1050F0000A4423F8152000F0D1F860B100F108034C
:10510000C8F8043018F0080F354B364A08BF13466C
:1051100046F837300FE0002346F83730324B1A7824
:1051200001321A7007E018F0080F2D4B2D4A08BF06
:10513000134646F8373008232370F4E415F0010FC6
:1051400022D02A4902230B700022294B1A70294BC6
:1051500024481860284C5C6098602848D8601A6120
:105160009A610D20264B1870FF23264803700838DB
:10517000037018300270244A13709F22234B1A7058
:1051800001230B70BDE8F88F15F0800F05D00D22BC
:105190001B4B1A708022403B1A7015F0020F06D08C
:1051A000184B1A78D2B21A700222083B1A7015F006
:1051B000100F0ED01022164B1A70BDE8F88F002089
:1051C0000146FFF7C3FBB1E628460021FFF7BEFB0F
:1051D000ACE6BDE8F88F00BF58FCFF1F7CFFFF1F47
:1051E000C8004000880040002AFDFF1F94200740AF
:1051F000BCFCFF1F0080FF1F6CFCFF1FC0FCFF1FDB
:10520000C0200740882007408C20074084200740AA
:105210008020074008B501F087FE00231B491A468D
:105220005A50C81842600833882BF9D1184B1A68B5
:1052300042F480221A60154BC3F30721154A1170FE
:10524000C3F30741143211701B0E04321370FF2395
:10525000343A137008321370783A13700123843291
:10526000137000216C3211707C3A137070220A4B5B
:105270001A704FF40072A3F241331A60102203F146
:10528000C04303F5C8231A7008BD00BF0080FF1F8C
:10529000348004409C20074049E400E072B60D4B86
:1052A0001A68B2FA82F30B2B02D962B6002070475B
:1052B0004FF00041D94022EA010206490A6062B675
:1052C000054903EBC303DB00C8180022CA50426043
:1052D000704700BFA48FFF1F008CFF1F08B50F4B46
:1052E000C31A0F4AA2FB03131B090B2B14D80D4A38
:1052F00012783AB10C4A127812F0FF0F02D0FFF781
:105300007DFB08BD72B6094A4FF0004121FA03F354
:1053100011681943116062B608BD00BF008CFF1F01
:10532000398EE3382AFDFF1F34FDFF1FA48FFF1FB6
:1053300010B5134B1B6853B9124B1B7813F0FF0FBA
:1053400018D00320FFF726FB0D4B1860A8B10C4BBB
:10535000186843885A1C03441C7A03889A4206D36F
:10536000FFF7BCFF0022064B1A60204610BD4280AA
:10537000204610BD4FF0FF3010BD4FF0FF3010BD84
:1053800040FDFF1F34FDFF1F08B50D4B1B6883B99F
:105390000C4B1B7813F0FF0F08D00320FFF7FAFA2D
:1053A000074B186028B94FF0FF3008BD4FF0FF30B1
:1053B00008BD034B1B685A881344187A08BD00BF08
:1053C00040FDFF1F34FDFF1F044B9888044B1B68F2
:1053D0001BB11A885B88D31A184470477CFFFF1FE3
:1053E00040FDFF1F2DE9F04704460122374B1A709C
:1053F0000E46002964D0DFF8E080DFF8E0909A469E
:10540000334FD8F8003083BB99F8003013F0FF0F0A
:1054100006D100222D4B1A704FF0FF30BDE8F08707
:1054200048F601450420FFF7D3FA07280AD80123DC
:105430008AF80030FFF732FFC8F80000A8B900234F
:105440008AF80030013D01D03B7833B10122204B76
:105450001A704FF0FF30BDE8F08700F097FC99F824
:10546000003013F0FF0FDDD1D3E700233B70D8F8F5
:1054700000104A88C2F14005AE4238BF354602F1FD
:1054800008030B442A444A80761B3DB1254414F896
:10549000012B03F8012BAC42F9D100E025464B88E3
:1054A0003F2B07D940230B800420FFF7EBFA0023A2
:1054B000C8F800300522074B1A700EB12C46A0E741
:1054C0000020024B1870BDE8F08700BF37FDFF1FBA
:1054D0003CFDFF1F36FDFF1F38FDFF1F34FDFF1F82
:1054E00000B583B002AB03F8010D18460121FFF7A8
:1054F00079FF03B05DF804FB10B5144B1B7813F073
:10550000FF0F21D00122124B1A70124B196851B1B2
:105510000024114B1C704B880B800420FFF7B2FA5B
:105520000C4B1C600DE0FFF7B9FE014630B10022C4
:10553000094B1A700420FFF7A5FA02E00122064B7E
:105540001A700022024B1A7010BD00BF34FDFF1FFD
:1055500037FDFF1F38FDFF1F36FDFF1F08B50E4B3F
:105560001B7813F0FF0F16D10C4B196841B14B8813
:105570000B800420FFF786FA0022084B1A6008BD52
:10558000FFF78CFE014618B10420FFF77BFA08BD37
:105590000122034B1A7008BD37FDFF1F38FDFF1FA6
:1055A00036FDFF1FF0B4C02928BFC02172B6134BCF
:1055B0001860134B00221A605A609A60DA601A6110
:1055C0005A61C1B113460E4C01275A0903F01F0658
:1055D00007FA06F654F82250354344F822500133B6
:1055E0008B42F2D10022134684186370013302F516
:1055F00082728B42F8D162B6F0BC704750FDFF1F3B
:1056000058FDFF1F10B472B6234B1B688BB9224B99
:105610005B6883B9204B9B687BB91F4BDB6873B910
:105620001D4B1B696BB91C4B5B6963B962B60020EB
:105630002EE0194A08E0194A06E0194A04E0194A1E
:1056400002E0194A00E0194AB3FA83F14FF0004032
:10565000C84023EA00031360154803780133DBB226
:10566000037062B60C48121A9210C1EB421202EBA0
:10567000821241F67C7101EB82020E49096888189A
:1056800001248C540C4A12789A423CBF0A4A137087
:105690005DF8044B704700BF58FDFF1F5CFDFF1F06
:1056A00060FDFF1F64FDFF1F68FDFF1F6CFDFF1FF6
:1056B00055FDFF1F50FDFF1F4CFDFF1F427872B6C6
:1056C0000378012B02D9013B037011E05111094B02
:1056D000D24302F01F024FF0004020FA02F253F8CA
:1056E0002100104343F82100034B1A78013A1A7045
:1056F00062B6704758FDFF1F55FDFF1F30B4C368E9
:1057000083B1187A90420AD158685C7A006950F8DF
:10571000245025B940F82410087801300870DB685F
:10572000002BEED130BC7047437A8B4206D9036917
:1057300053F82100002243F82120704700207047D1
:1057400038B5437A8B4218D9036953F821400022B7
:1057500043F821209CB12378012B12D9FFF752FF87
:10576000054628B10430211D4FF48072FEF71AFB64
:105770002378013B2370284638BD002038BD2046E1
:1057800038BD204638BD00BF4368427A5B7A9A42F2
:1057900010D872B60368DA680AB9D86004E0D36832
:1057A0000BB11A46FBE7D06002680123137242680E
:1057B000137262B6704700BF084B1B785BB9D022EA
:1057C000074B1A704FF08042A3F256331A60012043
:1057D000024B187070470020704700BF54FDFF1F38
:1057E0005EE400E0F8B5184B1A6842F080721A6067
:1057F000164B1A6842F001021A6004331F68144BFA
:105800001C689CB1134D237A6BB12E6823681B680A
:10581000204698472B689B1B1B099AB2A280E188FF
:105820008B4288BFE2806469002CECD1094B1B6875
:10583000DF1B3F09BBB2084A1380084A128897420F
:1058400084BF064A1380F8BDFCED00E0001000E0C4
:1058500048FDFF1F041000E070FDFF1F56FDFF1FF5
:1058600030B472B699B902688AB103790F2B0ED899
:1058700027490988194111F0010F08D003F100737D
:1058800003F59063B2EB431F01D162B63EE0204BBB
:105890001D882946002341FA03F212F0010F2DD191
:1058A000012202FA03F42543194A158062B6DAB2DE
:1058B000027118490C6844F002040C6004390C6849
:1058C00044F002040C60822413490C601A310A70FF
:1058D00004310A7006390A7007310A7003F1007347
:1058E00003F590635B01036000221A605A609A60BE
:1058F000DA601A615A619A61DA6107E00133102BAC
:10590000C9D162B6002303601023037130BC704715
:1059100072FDFF1F408004400080004003790F2B80
:1059200010D8094A137072B6084B0279012101FAA6
:1059300002F2198821EA02021A8062B6102303716A
:1059400000230360704700BF1A80004072FDFF1FF4
:10595000F8B506460F46144652B1002533681B6859
:10596000304617F8011B98470544013CF6D100E08A
:1059700000252846F8BD00BF00B583B0054B1B8845
:10598000ADF8043003685B6801A90222984703B0B0
:105990005DF804FB70B40000F0B58BB0164622B978
:1059A00003681B68C9B298472FE0012A08BF0A267E
:1059B00021B930228DF82520212417E021243746F3
:1059C000B1FBF6F506FB1515EDB22246092D94BF85
:1059D00030353735EDB20DF1280E724402F8245CF3
:1059E000B1FBF7F111B1013CE4B2E9E733B1013C9D
:1059F000E4B20AAB23442D2203F8242C03685B682D
:105A000001A92144C4F1220298470BB0F0BD00BFA8
:105A100008B50029BABF49422D2300230A22FFF707
:105A2000BBFF08BD10B4401A019CE41A04FB00F44B
:105A3000521A94FBF2F018445DF8044B704700BF13
:105A400010B50446006803F00BFD204610BD00BFF2
:105A500038B504460D460068013104F035FB18B135
:105A600020606560012038BD002038BD10B50446B7
:105A700043688B420AD2FFF7EBFF034648B1A368A5
:105A800033B9236800221A70012302E0012300E0E9
:105A90000123184610BD00BF70B504460E461546DA
:105AA0002AB9036803B11A700023A36012E01146FB
:105AB000FFF7DCFF48B9206818B103F0D1FC0023E0
:105AC000236000236360A36004E0A5602068314682
:105AD00004F082FE204670BD38B504460023036002
:105AE0004360836003730D4639B1084604F0D2FE6B
:105AF000024620462946FFF7CFFF204638BD00BFAB
:105B000008B50B46884203D009689A68FFF7C4FFBE
:105B100008BD00BF10B504460023036043608360E6
:105B20000373FFF7EDFF204610BD00BF38B50446F4
:105B30000D4641B1084604F0ADFE02462046294616
:105B4000FFF7AAFF01E000238360204638BD00BFB5
:105B500010B586B00446002303604360836003737E
:105B6000084601A900F056F9204601A9FFF7DEFF1B
:105B7000204606B010BD00BF70B504460D468368D0
:105B80005AB1D6183146FFF771FF30B12068A368CB
:105B90001844294604F020FEA660204670BD00BFD0
:105BA00008B50B4609689A68FFF7E6FF08BD00BF15
:105BB00038B504460D4639B1084604F06BFE02467E
:105BC00020462946FFF7D8FF204638BD10B582B0E1
:105BD00004468DF8041000238DF8053001A9012238
:105BE000FFF7CAFF204602B010BD00BF10B5044643
:105BF000FFF7ECFF204610BD08B5036813B1096834
:105C000059B906E00A6862B18B6863B11078404206
:105C100008BD82684AB1187808BD184604F0CEFC69
:105C200008BD002008BD002008BD002008BD00BF41
:105C300008B5836843B929B10878D0F1010038BFAD
:105C4000002008BD012008BD31B903681878D0F1E3
:105C5000010038BF002008BD006804F0AFFCD0F19F
:105C6000010038BF002008BD10B58B688468E41AB5
:105C700094420CD3006860B1096861B110441A46BF
:105C800004F038FED0F1010038BF002010BD002024
:105C900010BD002010BD002010BD00BF08B58268F7
:105CA0008B689A4203D30022FFF7DEFF08BD002075
:105CB00008BD00BF08B582688B689A420CD30068A3
:105CC00060B1096861B1D31A184404F077FCD0F1CF
:105CD000010038BF002008BD002008BD002008BD1D
:105CE000002008BD38B50C469AB191B1816899423F
:105CF00002D80023237038BD551EC91A8D4228BF13
:105D00000D460168204619442A4604F04DFE002342
:105D1000635538BD08B5006810B103F05DFB08BDE0
:105D2000002008BD08B5FBF74BF8FBF7D3FA00F0ED
:105D30002DF8FAE708B5FFF747FB08BD08B5FFF7F0
:105D4000F7FA08BD08B5FFF71FFB08BD08B5FFF758
:105D5000D3FB08BD08B50846FFF7C2FB08BD00BF6E
:105D600008B508461146FFF73DFB08BD704700BF68
:105D7000044B00221A714FF47A7199601A73024A27
:105D80001A60704778FDFF1F80B4000008B50F4B04
:105D90001B78CBB901220D4B1A70FFF715FB08B128
:105DA000FFF7E4FF00F034FA08B101F087F900F0E2
:105DB0002DFD08B101F018FA00F0CCFF08B101F098
:105DC000A9FA0022014B1A7008BD00BF88FDFF1F11
:105DD00030B40023B0FBF2F402FB14041D46092C7E
:105DE00094BF30343734E4B2CC54B0FBF2F008B195
:105DF0000133EFE70D4400226A70934207DD885CAF
:105E0000CC5C8C54C8540132013B9A42F7DB084603
:105E100030BC704710B50C46002802DBFFF7D8FFF6
:105E200010BD2D2301F8013B4042FFF7D1FF204672
:105E300010BD00BF194B1A6842F480621A6000233B
:105E4000174A1370174A1370174A1370174A1370C2
:105E5000174A137040F21332164B1A604FF4517206
:105E600004331A60C0F34432134B1A70C0F3471264
:105E70005A7000F01F00987204229A700221D9749F
:105E80005A7588221A743C22DA7040220B4B1A7021
:105E90004FF40052A3F229331A6070473480044053
:105EA00014FEFF1F91FDFF1F1CFEFF1F15FEFF1FAD
:105EB00090FDFF1F40A0044000A006402DE400E03C
:105EC000164B9B7803F0EC0300F00302134310F031
:105ED000040F18BF43F01003104A937000F00F0333
:105EE000042B04D11346927942F040029A710B4B75
:105EF0005A7902F0EF0210F0100F18BF42F01002B2
:105F0000064B5A719B7903F0EF0310F0200F18BF76
:105F100043F01003014A9371704700BF00A0064090
:105F200010B5144B1B6813F4806F21D0124B1B78F3
:105F300013F0FF0F06D0104CFFF728FF237813F063
:105F4000FF0FF9D14FF400520C4B1A6000230C4A9A
:105F5000D37040F203120B490A6004310A600A4A06
:105F600013700A4A13700A4B1B680BB101221A7096
:105F700010BD00BF3480044090FDFF1F84E100E0AD
:105F800000A0064040A0044014FEFF1F91FDFF1F2B
:105F90008CFDFF1F10B50446094A137813F0FF0F5C
:105FA000FBD120460121FEF71BFC20460021FEF715
:105FB000E5FB044B53F83420034B1A6010BD00BFBF
:105FC00090FDFF1F60B3000018FEFF1F10B50D4BC2
:105FD0001B6813F4806F12D021280CD80A4C0B4B8D
:105FE00053F8303023600121FEF7FAFB23680022CA
:105FF0001A70012010BD0020034B186010BD002056
:1060000010BD00BF348004408CFDFF1F60B3000052
:10601000114B1B6813F4806F1BD0122804D140F27F
:1060200002320E4B1A600DE0142804D140F2023205
:106030000B4B1A6006E00B4B5A7B02F0FE025A73C0
:1060400000207047074B5A7B42F001025A7301202F
:1060500070470020704700BF348004400CA004400B
:1060600014C0044000A006402DE9F04107461F4B34
:106070001B6813F4806F37D01D4B1B680BB10122D6
:106080001A701C4B1C780134402C28BF00241A4D78
:106090001A4EDFF86C8017E0FEF778F940280FDC25
:1060A000337913F0800F0FD02B780133402B28BFAA
:1060B000002318F80320D2B2F271DBB22B7003E098
:1060C000FF2801DDFFF762FE2B78DBB29C42E3D0B4
:1060D000FFB20B4B1F5501220A4B1A70E4B2054B5D
:1060E0001C70BC22054BDA70BDE8F081348004409E
:1060F00018FEFF1F1CFEFF1F15FEFF1F00A006401D
:1061000094FDFF1F90FDFF1F2DE9F84F0746284B18
:106110001B6813F4806F49D0264B1B680BB101221A
:106120001A7007EB010B5F453DD2DFF89890224EC5
:10613000DFF88C80DFF890A099F800400134402C03
:1061400028BF00243578EDB2A54220D1BC2388F8C1
:106150000330FEF71BF9402811DC98F8043013F0E7
:10616000800F10D033780133402B28BF00231AF85A
:106170000320D2B288F80720DBB2337003E0FF2897
:1061800001DDFFF703FE3378DBB29D42E1D017F863
:10619000013B0AF804300122084B1A70E4B289F876
:1061A00000405F45C8D1BC22054BDA70BDE8F88FCE
:1061B0003480044018FEFF1F15FEFF1F90FDFF1FD7
:1061C00000A006401CFEFF1F94FDFF1F10B5064BEC
:1061D0001B7813F0FF0F06D0034CFFF7D7FD237891
:1061E00013F0FF0FF9D110BD90FDFF1F064B1B7878
:1061F000DBB2064A1278D2B293422CBF3F3202F190
:10620000FF32D01A704700BF1CFEFF1F15FEFF1F94
:10621000054B1878C0B2054B1B78DBB2984238BFEB
:106220004030C01A704700BF14FEFF1F91FDFF1FD2
:1062300010B4184B1A78D2B2174B1B78DBB29A42C3
:1062400018D001333F2B18D81449C85CC0B2DCB257
:1062500011490C7012490968C9B19A4203D300E090
:106260000023D31A01E04032D31A1A2B0FDC00238B
:106270000B700CE04FF0FF3009E0084B1878C0B20B
:106280000021054B1970064B19680029E8D15DF80B
:10629000044B704714FEFF1F91FDFF1FD4FDFF1F2D
:1062A0008CFDFF1F094B1A78D2B2094B1B78DBB269
:1062B0009A4207D00133402B28BF0023054AD05C07
:1062C000C0B270474FF0FF30704700BF14FEFF1F91
:1062D00091FDFF1FD4FDFF1F0D4B1B6813F4806F52
:1062E00014D00C4BDA7802F0CB02DA7040225A74E8
:1062F000DA7842F03402DA70074B1A78D2B2074BE0
:106300001A70074B1B680BB100221A70704700BF50
:106310003480044000A0064091FDFF1F14FEFF1FC3
:106320008CFDFF1F70B43D4B1B7913F0300F33D041
:1063300072B63A4B9B7D03F0FF022BB9374BDA79EB
:1063400040225A7462B627E062B6354B1978C9B25A
:10635000344B1C78E4B2314D334EEB79D8B24B1C40
:10636000402B28BF0023A3421CBFF0541946531EE4
:1063700013F0FF02F1D1CAB2294B1A702B4B1B68E4
:1063800053B1A1422EBFC4EB0101C4F1400409196D
:106390002729C4BF01221A70204BDA78D2B212F03A
:1063A000800F27D01B7913F0800F23D0204B1C784F
:1063B000E4B2204B1B78DBB29C4210D017491E4D33
:1063C00001E0A3420BD00133402B28BF0023087902
:1063D000E85CC0B2C871087DC0B20728F1D9DBB251
:1063E00014490B700D4B1B7913F0800F02D07C21E8
:1063F0000A4BD97012F0400F0ED0084B1B7913F0E6
:10640000400F09D000220D4B1A700D4B1B6803B1D1
:106410001A703C22014BDA7070BC704700A0064035
:1064200014FEFF1F91FDFF1FD4FDFF1F8CFDFF1FFA
:106430001CFEFF1F15FEFF1F94FDFF1F90FDFF1F99
:1064400018FEFF1F194B1A6842F400621A600023FD
:10645000174A1370174A1370174A1370174A1370AC
:10646000174A137040F21332164B1A604FF45172F0
:1064700004331A60C0F34432134B1A70C0F347124E
:106480005A7000F01F00987204229A700221D97489
:106490005A7588221A743C22DA7040220B4B1A700B
:1064A0004FF40042A3F22B331A607047348004404B
:1064B00090FEFF1F25FEFF1F98FEFF1F91FEFF1F8E
:1064C00024FEFF1F0CB0044000B006402FE400E0A3
:1064D000164B9B7803F0EC0300F00302134310F01B
:1064E000040F18BF43F01003104A937000F00F031D
:1064F000042B04D11346927942F040029A710B4B5F
:106500005A7902F0EF0210F0100F18BF42F010029B
:10651000064B5A719B7903F0EF0310F0200F18BF60
:1065200043F01003014A9371704700BF00B006406A
:1065300010B5144B1B6813F4006F21D0124B1B785D
:1065400013F0FF0F06D0104CFFF720FC237813F058
:10655000FF0FF9D14FF400420C4B1A6000230C4A94
:10656000D37040F203120B490A6004310A600A4AF0
:1065700013700A4A13700A4B1B680BB101221A7080
:1065800010BD00BF3480044024FEFF1F84E100E002
:1065900000B006400CB0044090FEFF1F25FEFF1F18
:1065A00020FEFF1F10B50446094A137813F0FF0FB1
:1065B000FBD120460121FEF713F920460021FEF70A
:1065C000DDF8044B53F83420034B1A6010BD00BFB4
:1065D00024FEFF1F60B3000094FEFF1F10B50D4B9B
:1065E0001B6813F4006F12D021280CD80A4C0B4BF7
:1065F00053F8303023600121FEF7F2F823680022BF
:106600001A70012010BD0020034B186010BD00203F
:1066100010BD00BF3480044020FEFF1F60B30000A7
:106620000D4B1B6813F4006F13D017280AD140F2EA
:1066300002320A4B1A600A4B5A7B42F001025A732B
:1066400001207047064B5A7B02F0FE025A7300206D
:1066500070470020704700BF3480044008B00440F9
:1066600000B006402DE9F04107461F4B1B6813F4AC
:10667000006F37D01D4B1B680BB101221A701C4BE9
:106680001C780134282C28BF00241A4D1A4EDFF83C
:106690006C8017E0FDF77AFE40280FDC337913F0A9
:1066A000800F0FD02B780133282B28BF002318F838
:1066B0000320D2B2F271DBB22B7003E0FF2801DDC0
:1066C000FFF764FB2B78DBB29C42E3D0FFB20B4BAD
:1066D0001F5501220A4B1A70E4B2054B1C70BC22F4
:1066E000054BDA70BDE8F0813480044094FEFF1F52
:1066F00098FEFF1F91FEFF1F00B0064028FEFF1FFF
:1067000024FEFF1F2DE9F84F0746284B1B6813F4A2
:10671000006F49D0264B1B680BB101221A7007EBA2
:10672000010B5F453DD2DFF89890224EDFF88C8058
:10673000DFF890A099F800400134282C28BF0024ED
:106740003578EDB2A54220D1BC2388F80330FDF79F
:106750001DFE402811DC98F8043013F0800F10D093
:1067600033780133282B28BF00231AF80320D2B234
:1067700088F80720DBB2337003E0FF2801DDFFF764
:1067800005FB3378DBB29D42E1D017F8013B0AF8F4
:1067900004300122084B1A70E4B289F800405F45CA
:1067A000C8D1BC22054BDA70BDE8F88F34800440B4
:1067B00094FEFF1F91FEFF1F24FEFF1F00B0064046
:1067C00098FEFF1F28FEFF1F10B5064B1B7813F025
:1067D000FF0F06D0034CFFF7D9FA237813F0FF0F11
:1067E000F9D110BD24FEFF1F064B1B78DBB2064A11
:1067F0001278D2B293422CBF273202F1FF32D01A64
:10680000704700BF98FEFF1F91FEFF1F054B1878D1
:10681000C0B2054B1B78DBB2984238BF4030C01A7B
:10682000704700BF90FEFF1F25FEFF1F10B4184BDE
:106830001A78D2B2174B1B78DBB29A4218D00133C8
:106840003F2B18D81449C85CC0B2DCB211490C7097
:1068500012490968C9B19A4203D300E00023D31A50
:1068600001E04032D31A1A2B0FDC00230B700CE02E
:106870004FF0FF3009E0084B1878C0B20021054BFB
:106880001970064B19680029E8D15DF8044B704770
:1068900090FEFF1F25FEFF1F50FEFF1F20FEFF1F63
:1068A000094B1A78D2B2094B1B78DBB29A4207D057
:1068B0000133402B28BF0023054AD05CC0B270478B
:1068C0004FF0FF30704700BF90FEFF1F25FEFF1FF7
:1068D00050FEFF1F0D4B1B6813F4006F14D00C4BC0
:1068E000DA7802F0CB02DA7040225A74DA7842F099
:1068F0003402DA70074B1A78D2B2074B1A70074B82
:106900001B680BB100221A70704700BF348004402E
:1069100000B0064025FEFF1F90FEFF1F20FEFF1F58
:1069200070B43D4B1B7913F0300F33D072B63A4B35
:106930009B7D03F0FF022BB9374BDA7940225A7462
:1069400062B627E062B6354B1978C9B2344B1C7871
:10695000E4B2314D334EEB79D8B24B1C402B28BFFB
:106960000023A3421CBFF0541946531E13F0FF022C
:10697000F1D1CAB2294B1A702B4B1B6853B1A142FB
:106980002EBFC4EB0101C4F1400409192729C4BF7B
:1069900001221A70204BDA78D2B212F0800F27D081
:1069A0001B7913F0800F23D0204B1C78E4B2204BCE
:1069B0001B78DBB29C4210D017491E4D01E0A34268
:1069C0000BD00133282B28BF00230879E85CC0B224
:1069D000C871087DC0B20728F1D9DBB214490B7029
:1069E0000D4B1B7913F0800F02D07C210A4BD9701C
:1069F00012F0400F0ED0084B1B7913F0400F09D056
:106A000000220D4B1A700D4B1B6803B11A703C220B
:106A1000014BDA7070BC704700B0064090FEFF1F5B
:106A200025FEFF1F50FEFF1F20FEFF1F98FEFF1FC9
:106A300091FEFF1F28FEFF1F24FEFF1F94FEFF1F75
:106A4000174B1A6842F480521A600023154A1370DB
:106A5000154A1370154A1370154A1370154A1370AE
:106A600040F21331144A11604FF451710432116035
:106A7000C0F34431114A1170C0F34711517000F056
:106A80001F009072937013742C23D37040220C4B10
:106A90001A704FF40032A3F22D331A60704700BF12
:106AA000348004400CFFFF1FA1FEFF1F14FFFF1FD7
:106AB0000DFFFF1FA0FEFF1F08C0044000C00640DE
:106AC00031E400E0164B9B7803F0EC0300F0030286
:106AD000134310F0040F18BF43F01003104A9370D3
:106AE00000F00F03042B04D11346927942F04002C8
:106AF0009A710B4B5A7902F0EF0210F0100F18BF89
:106B000042F01002064B5A719B7903F0EF0310F02C
:106B1000200F18BF43F01003014A9371704700BF64
:106B200000C0064010B5144B1B6813F4805F21D0E1
:106B3000124B1B7813F0FF0F06D0104CFFF726F90D
:106B4000237813F0FF0FF9D14FF400320C4B1A6089
:106B500000230C4AD37040F203120B490A6004313F
:106B60000A600A4A13700A4A13700A4B1B680BB179
:106B700001221A7010BD00BF34800440A0FEFF1F28
:106B800084E100E000C0064008C004400CFFFF1F85
:106B9000A1FEFF1F9CFEFF1F10B50446094A137893
:106BA00013F0FF0FFBD120460121FDF719FE20460F
:106BB0000021FDF7E3FD044B53F83420034B1A602A
:106BC00010BD00BFA0FEFF1F60B3000010FFFF1F3D
:106BD00010B50D4B1B6813F4805F12D021280CD820
:106BE0000A4C0B4B53F8303023600121FDF7F8FDC0
:106BF000236800221A70012010BD0020034B18608A
:106C000010BD002010BD00BF348004409CFEFF1F5B
:106C100060B300000D4B1B6813F4805F13D00E2887
:106C20000AD140F202320A4B1A600A4B5A7B42F0F8
:106C300001025A7301207047064B5A7B02F0FE0294
:106C40005A73002070470020704700BF3480044012
:106C500004C0044000C006402DE9F04107461F4B28
:106C60001B6813F4805F37D01D4B1B680BB10122EA
:106C70001A701C4B1C780134282C28BF00241A4D94
:106C80001A4EDFF86C8017E0FDF780FB40280FDC20
:106C9000337913F0800F0FD02B780133282B28BFC6
:106CA000002318F80320D2B2F271DBB22B7003E09C
:106CB000FF2801DDFFF76AF82B78DBB29C42E3D0B6
:106CC000FFB20B4B1F5501220A4B1A70E4B2054B61
:106CD0001C70AC22054BDA70BDE8F08134800440B2
:106CE00010FFFF1F14FFFF1F0DFFFF1F00C0064016
:106CF000A4FEFF1FA0FEFF1F38B505460C4629B1B4
:106D000015F8010BFFF7A8FF013CF9D138BD00BF12
:106D100010B5064B1B7813F0FF0F06D0034CFFF79E
:106D200035F8237813F0FF0FF9D110BDA0FEFF1F37
:106D3000064B1B78DBB2064A1278D2B293422CBFC4
:106D4000273202F1FF32D01A704700BF14FFFF1F35
:106D50000DFFFF1F054B1878C0B2054B1B78DBB247
:106D6000984238BF4030C01A704700BF0CFFFF1F69
:106D7000A1FEFF1F10B4184B1A78D2B2174B1B7824
:106D8000DBB29A4218D001333F2B18D81449C85CA3
:106D9000C0B2DCB211490C7012490968C9B19A42FB
:106DA00003D300E00023D31A01E04032D31A1A2B98
:106DB0000FDC00230B700CE04FF0FF3009E0084BB4
:106DC0001878C0B20021054B1970064B19680029CC
:106DD000E8D15DF8044B70470CFFFF1FA1FEFF1FB9
:106DE000CCFEFF1F9CFEFF1F094B1A78D2B2094B45
:106DF0001B78DBB29A4207D00133402B28BF002317
:106E0000054AD05CC0B270474FF0FF30704700BFFA
:106E10000CFFFF1FA1FEFF1FCCFEFF1F054B1A78C2
:106E2000D2B2054B1A70054B1B680BB100221A70C9
:106E3000704700BFA1FEFF1F0CFFFF1F9CFEFF1F3E
:106E40002F4B1B7913F0200F23D02D4BDB79D9B2B8
:106E50002C4B1B780133402B28BF00232A4A127881
:106E6000D2B29A4204D0294AD154D9B2254A1170DB
:106E7000274A116869B1274A1278D2B293422EBFCD
:106E8000C2EB0303C2F140029B18272BC4BF0123AE
:106E90000B701B4BDB78DBB213F0800F1CD0184A51
:106EA000127912F0800F17D01B4A1178C9B2194A13
:106EB0001278D2B2914203D16C21114AD1700BE009
:106EC0000132282A28BF00221449885CC0B20C492C
:106ED000C871D2B20F490A7013F0400F0ED0084BA0
:106EE0001B7913F0400F09D000220D4B1A700D4B87
:106EF0001B6803B11A702C22014BDA70704700BF77
:106F000000C006400CFFFF1FA1FEFF1FCCFEFF1FAD
:106F10009CFEFF1F0DFFFF1F14FFFF1FA4FEFF1F9E
:106F2000A0FEFF1F10FFFF1F00B585B072B61B4B00
:106F300070221A7041211A4A11700F21013A117002
:106F400080221A701A46137813F0800FFBD0154B6D
:106F5000186862B6144B98429CBF00EB800040005A
:106F600001A90A22FEF734FF9DF804307BB908E03E
:106F700001A9595C31B19180023201330A2BF7D15A
:106F800000E0002301335B00084A137003E0074A66
:106F900053800123ECE705B05DF804FB00000240DC
:106FA00007000240080002407F9698003490FF1FBF
:106FB00008B503681B68C9B2984708BD08B50368DF
:106FC0001B68C9B2984708BD08B503681B68C9B2F9
:106FD000984708BD08B503681B68C9B2984708BD43
:106FE00008B5044800EB5100B0FBF1F0FEF722FFBA
:106FF00008BD00BF0044950810B51446054800EBD5
:107000005100B0FBF1F0FEF715FF2046FEF758FFE8
:1070100010BD00BF0044950808B5FEF781FF08BD0C
:1070200008B50846FEF7B6FF08BD00BF08B508461C
:10703000FEF7CCFF003018BF012008BD08B5084698
:10704000FEF7E6FF003018BF012008BD08B5FFF7C6
:10705000DFF808BD08B5FFF725F908BD08B5FFF74B
:10706000E7F808BD08B5FFF7B1F808BD08B5FFF7A8
:1070700033F908BD08B5FFF7B9F808BD08B50846EB
:10708000FEF7F2FF012008BD08B50846FEF7ECFF49
:10709000012008BD10B5144608461146FFF734F824
:1070A000204610BD38B50D46084603F0F3FB0446F4
:1070B00028462146FFF728F8204638BD704700BF14
:1070C000044B00221A714FF47A7199601A73024AC4
:1070D0001A60704718FFFF1FF8B4000008B5036876
:1070E0001B68C9B2984708BD08B503681B68C9B2D8
:1070F000984708BD08B503681B68C9B2984708BD22
:1071000008B503681B68C9B2984708BD08B50448AC
:1071100000EB5100B0FBF1F0FFF794F908BD00BFA0
:107120000044950810B51446054800EB5100B0FB2B
:10713000F1F0FFF787F92046FFF7CAF910BD00BF4D
:107140000044950808B5FFF7F3F908BD08B50846EF
:10715000FFF728FA08BD00BF08B50846FFF73EFA5A
:10716000003018BF012008BD08B50846FFF758FADF
:10717000003018BF012008BD08B5FFF747FB08BD68
:1071800008B5FFF78DFB08BD08B5FFF74FFB08BD3D
:1071900008B5FFF719FB08BD08B5FFF79BFB08BD55
:1071A00008B5FFF721FB08BD08B50846FFF75AFAF6
:1071B000012008BD08B50846FFF754FA012008BDB4
:1071C00010B5144608461146FFF79CFA204610BD3C
:1071D00038B50D46084603F05DFB044628462146B7
:1071E000FFF790FA204638BD704700BF044B0022DD
:1071F0001A714FF47A7199601A73024A1A607047D3
:1072000028FFFF1F50B5000008B503681B68C9B20E
:10721000984708BD08B503681B68C9B2984708BD00
:1072200008B503681B68C9B2984708BD08B503686C
:107230001B68C9B2984708BD08B5044800EB510067
:10724000B0FBF1F0FFF7FCFB08BD00BF00A24A0451
:1072500010B51446054800EB5100B0FBF1F0FFF704
:10726000EFFB2046FFF72EFC10BD00BF00A24A0432
:1072700008B5FFF757FC08BD08B50846FFF78CFCBA
:1072800008BD00BF08B50846FFF7A2FC003018BFD4
:10729000012008BD08B50846FFF7BCFC003018BF48
:1072A000012008BD08B5FFF755FD08BD08B5FFF77B
:1072B0009BFD08BD08B5FFF75DFD08BD08B5FFF7EC
:1072C00027FD08BD08B5FFF7A9FD08BD08B5FFF704
:1072D0002FFD08BD08B50846FFF7BEFC012008BD1C
:1072E00008B50846FFF7B8FC012008BD10B51446E4
:1072F00008461146FFF700FD204610BD38B50D4683
:10730000084603F0C7FA044628462146FFF7F4FC76
:10731000204638BD704700BF044B00221A714FF45D
:107320007A7199601A73024A1A60704738FFFF1F1A
:10733000A8B500002DE9F04FDFF8B8A28BB01D46CC
:1073400080468946144600F073F99AF900300133FB
:1073500006460F4604D02046294600F06FFF20B9AC
:10736000304639460BB0BDE8F08F4046494600F044
:1073700065FF834600282CD12046294600220023A1
:1073800001F0D0FC0028EBD0944B9AF900109448FF
:10739000CDF820B000220126CDE906234B1CCDE913
:1073A0000289CDE90445009601900DD002290BD049
:1073B000684600F06BFF002800F09580089B1BB129
:1073C00002F018F8089B0360DDE906010BB0BDE888
:1073D000F08F002200234046494601F0A3FCF8B19B
:1073E000204629460022002301F09CFC8346002809
:1073F0004DD07B4A9AF900300192CDE90445012134
:10740000002200240025CDE90289CDE9064500913E
:107410000892002BCCD0714B0022CDE90623D3E794
:107420003046394600F004FF8346002860D0002231
:1074300000233046394601F075FC002890D04046C4
:10744000494600F0F5FE00288AD02046294600F083
:10745000EFFE002884D09AF90030614A0192CDE90C
:1074600004450421002200240025022BCDE90289D5
:10747000CDE906450091089200F08280684600F050
:1074800005FF00287CD0089B002B9DD098E7204664
:10749000294600F0CDFE00283FF462AF2046294681
:1074A0000022002301F048FC00283FF459AF4C4B68
:1074B0009AF80010CDF820B001228DE80C00CDE93B
:1074C0000289CDE904450022002934D10023CDE909
:1074D0000623684600F0DAFE0028D4D101F08AFFC6
:1074E00021230360CFE701F085FF2123036065E7D7
:1074F0004046494600F09CFE002898D02046294688
:1075000000F096FE002892D03046394600F096FEF4
:10751000B8B9334B9AF8006008900122CDE902898E
:10752000CDE904458DE80C00002E2ED10024002565
:10753000CDE90645CDE72B4B0229CDE90623CDD079
:10754000C7E7274A9AF90030CDF820B003218DE82B
:107550000600CDE90289CDE90445404649460022AE
:10756000F3B9214F4FF060460023CDE9066701F0E3
:10757000E3FB002840D19AF90030022B7FF47EAF64
:1075800001F038FF222303607DE70020002102463E
:107590000B4601F089FA022ECDE906019ED098E74C
:1075A000124F00260023CDE9066701F0C5FB002835
:1075B000E1D000220E4B2046294601F04BF904464B
:1075C0000D4600F06BFE22462B4601F0ABFB002877
:1075D000D1D1044B0022CDE90623CCE70000F03FD7
:1075E000F8B500000000F0FFFFFFEF470000F07F5C
:1075F0000000E03F4C90FF1F00220A4B2046294626
:1076000001F028F904460D4600F048FE22462B46BC
:1076100001F088FB0028AED1034B4FF06042CDE96A
:107620000623A8E70000E03FFFFFEFC7FFFFFFFFD3
:107630002DE9F04F23F0004B91B089460F465BEAED
:107640000201CDE9022314461D46804606462ED08F
:10765000634B29F0004A9A4522DC1FD0604B9B45C2
:107660001EDC77D0002F78DB0022049264BB5C4BD9
:107670009B4500F091805B4B9B4565D0B5F1804FF9
:1076800000F0F783584B9D421ED1002F1CDB404673
:10769000494611B0BDE8F04F00F006BD0028DDD02E
:1076A0000AF1404A0AF5801A5AEA060A04D14D49FD
:1076B000002011B0BDE8F08F4C4811B0BDE8F04F8C
:1076C00000F0E6BD002104914046494600F0ACFDC3
:1076D000E6B9BAF1000F04D0424B27F040429A427B
:1076E00014D1002DC0F20584002FE2DA0AF1404ADD
:1076F000DDF810B00AF5801A5BEA0A0B5ED0049A36
:10770000012AD6D101F100431946D2E7FB0F03F15C
:10771000FF3C049B53EA0C034ED0354B9B456DDD7B
:1077200003F104739B4540F3EC83324B9A4540F3DD
:107730009A83002D40F39A8327A1D1E900010246E4
:107740000B4601F087F8B4E7002DC0F248844046AC
:107750004946AEE7002C85D0A2E7274B9B4536DC97
:10776000A3F154739B4540F38B834FEA2B5340F2B4
:107770001342934240F34984C3F58663033324FAEA
:1077800003F202FA03F3A3427FF46EAF02F00102A8
:10779000C2F10202049269E70AF1404303F5801343
:1077A000334384D0134B9A4540F39B83002DC0F2A2
:1077B0005D83DDE902017CE74046494602460B460F
:1077C00000F094FE02460B4601F06EF971E70223C9
:1077D00004934BE7AFF300809C7500883CE4377E50
:1077E0000000F07F0000F03F0000E03FF4AE00003A
:1077F0000000E041FFFFEF3FFFFF3F43BAF5801F6E
:1078000080F2EB83AA4BCDF804C0002201F022F8ED
:10781000DDF804C08A466FF034034FEA2A55A54AC2
:10782000CAF3130AA5F2FF354AF07F541D4492456E
:107830000F9544F4401440F3CD839F4B9A4540F399
:10784000FA83DDF83CA000250AF1010ACDF83CA03E
:10785000A4F580142B46994ACDF804C0DB000E93A2
:107860001344D3E90067214632463B46CDE90A017D
:1078700000F03CFE3246804689463B46DDE90A017F
:1078800000F036FE02460B4600208D4901F00CF94F
:10789000CDE90C01DDE90C234046494600F0DAFF52
:1078A000CDE906016110DDE906AB41F0005101F5BB
:1078B00000214B190021CDE908AB0891DDE908ABA7
:1078C00000225046594614461D4600F0C3FF0246AA
:1078D0000B464046494600F009FE3246804689463E
:1078E0003B462046294600F001FE02460B46DDE9F4
:1078F0000A0100F0FBFD02460B465046594600F0D7
:10790000A9FF02460B464046494600F0EFFDDDE97F
:107910000C2300F09FFF06460F46DDE906010246F4
:107920000B4600F097FF02460B4604460D4600F05A
:1079300091FF4FA3D3E9002380468946204629467C
:1079400000F088FF4CA3D3E9002300F0D1FD2246CC
:107950002B4600F07FFF4AA3D3E9002300F0C8FDC7
:1079600022462B4600F076FF47A3D3E9002300F020
:10797000BFFD22462B4600F06DFF45A3D3E900234F
:1079800000F0B6FD22462B4600F064FF42A3D3E987
:10799000002300F0ADFD02460B464046494600F08C
:1079A00059FFDDE9062304460D465046594600F0CE
:1079B0009FFD32463B4600F04DFF22462B4600F02D
:1079C00097FD5246804689465B465046594600F030
:1079D00041FF00223B4BCDE90A0100F089FD424600
:1079E0004B4600F085FD08980D46044622462B467E
:1079F0005046594600F02EFF224682468B462B46C3
:107A00003046394600F026FF002206460F46204643
:107A100029462C4B00F06AFDDDE90A2300F066FDE3
:107A200002460B464046494600F060FDDDE906236C
:107A300000F010FF02460B463046394600F058FD74
:107A40008046894642464B465046594600F050FD16
:107A5000089813A3D3E9002304460D4600F0FAFE6C
:107A600011A3D3E90023CDE90601204629462BE0E6
:107A7000EF4E454A287ECA3F65DBC9934A86CD3F13
:107A800001411DA96074D13F4D268F515555D53FF9
:107A9000FFAB6FDBB66DDB3F033333333333E33F91
:107AA000000000E009C7EE3FF5015B14E02F3EBE89
:107AB000000040438E98030079B60B0020B600000A
:107AC0000000F03F0000084000F0C4FE52460646A9
:107AD0000F465B462046294600F008FD02460B464D
:107AE0004046494600F002FD9FA3D3E9002300F081
:107AF000B1FE02460B463046394600F0F9FCDDF88F
:107B000038A0AB4B5344D3E9002300F0F1FC064608
:107B10000F980F4600F038FEA64B5344D3E900AB54
:107B200004460D4632463B46DDE9060100F0E0FC26
:107B300052465B4600F0DCFC22462B4600F0D8FCA7
:107B4000089822462B468046894600F0CFFC5246D4
:107B50005B4600F0CBFCDDE9062300F0C7FC0246E3
:107B60000B463046394600F0C1FCDDF804C08246C1
:107B70008B4604994B1E53EA0C030CBF8E4B8F4B64
:107B80000022CDE90823DDE90223CDE90423002307
:107B90000493DDE90445DDE902012B46224600F0AD
:107BA000A5FC42464B4600F055FE524606460F469F
:107BB0005B46DDE9020100F04DFE02460B46304611
:107BC000394600F095FC42464B4682468B4620469D
:107BD000294600F03FFE06460F463B4650465946B2
:107BE000324600F085FC764B9942804689460D4628
:107BF00040F34A8101F13F4303F5E003034340F0C2
:107C0000F6815BA3D3E900235046594600F070FC8F
:107C10003246CDE902013B464046494600F066FC4B
:107C200002460B46DDE9020101F0A4F8002840F00D
:107C3000DE81CC464FEA2C53A3F2FE334FF4801082
:107C400018412844C0F30A515E4AA1F2FF3342FAB8
:107C500003FEC1F58261C0F3130420EA0E03033171
:107C600044F4801040FA01F1002D0491BCBF494258
:107C7000049100223046394600F038FC06460F4693
:107C80003246504659463B4600F032FC049A1205F3
:107C90000292002438A3D3E9002320460D4600F0C9
:107CA000D9FD3246804689463B462046294600F0AB
:107CB0001DFC02460B465046594600F017FC30A307
:107CC000D3E9002300F0C6FD2FA3D3E90023064625
:107CD0000F462046294600F0BDFD02460B463046C1
:107CE000394600F005FC06460F4632463B46404604
:107CF000494600F0FDFB42464B4604460D4600F067
:107D0000F5FB02460B463046394600F0EFFB2246B3
:107D100082468B4620462B46294600F09BFD1CA33D
:107D2000D3E9002306460F4600F094FD1AA3D3E9D9
:107D3000002300F0DBFB32463B4600F08BFD18A32E
:107D4000D3E9002300F0D4FB32463B4600F082FD2D
:107D500015A3D3E9002300F0C9FB32463B4600F0EF
:107D600079FD31E0AFF30080FD033ADC09C7EE3F57
:107D7000FE822B654715973C00000000432EE63F2E
:107D8000EF39FAFE422EE63F396CA80C615C20BE4A
:107D9000D0A4BE726937663EF16BD2C541BDBB3E11
:107DA0002CDE25AF6A56113F93BDBE166CC1663FEF
:107DB00010B6000000B600000000F0BF0000F03F69
:107DC000FFFF8F40FFFF0F00A3A3D3E9002300F0C4
:107DD0008FFB32463B4600F03DFD02460B462046F7
:107DE000294600F083FB06460F4632463B462046B6
:107DF000294600F02FFD002280468946304639464C
:107E00004FF0804300F072FB02460B464046494665
:107E100000F04AFE524606460F4620465B4629467B
:107E200000F018FD52465B4600F062FB02460B462E
:107E30003046394600F05AFB22462B4600F056FBEE
:107E400002460B460020924900F050FB029C0C4475
:107E5000B4F5801F0246C0F2F2802346DDE9080136
:107E600000F0F8FC25E4002DFFF666AC00200021B0
:107E70001FE44046494642464B4600F0EBFC18E4FE
:107E800000210491FFF7F2BB824B21F0004C9C458E
:107E900040F3CA8001F17D5303F53C1303F55053C1
:107EA000034310D132463B46CDF804C000F01EFB20
:107EB00002460B465046594600F048FFDDF804C024
:107EC00000283FF4B7AEDDE9080165A3D3E900233C
:107ED00000F0C0FC62A3D3E9002300F0BBFCFFF775
:107EE000E8BB002DC2DA039B029803F10041FFF7C3
:107EF000E0BB02460B460020654900F0D5FDFFF7C8
:107F0000F3BB654B9A45AEDD614B9A453FF711AC2B
:107F100000225F4BCDF804C000F0E8FA52A3D3E989
:107F2000002304460D4600F095FC51A3D3E900233D
:107F300006460F462046294600F08CFC2246824623
:107F40008B462B462046294600F084FC00228046C2
:107F5000894620462946514B00F07CFC02460B46E0
:107F600045A1D1E9000100F0C1FA22462B4600F0FC
:107F700071FC02460B460020494900F0B7FA024660
:107F80000B464046494600F065FC3DA3D3E900237B
:107F900000F060FC02460B465046594600F0A6FA37
:107FA00004460D4622462B463046394600F0A0FADC
:107FB000002032463B468046894600F097FA02464A
:107FC0000B462046294600F091FADDF804C08246AF
:107FD0008B46CEE500252B463DE400231DE44246BA
:107FE0004B4600202A4900F05FFDFFF762BBDDE948
:107FF000080125A3D3E9002300F02CFC22A3D3E938
:10800000002300F027FCFFF754BB002C7FF45AAB91
:10801000C3F5826303334BFA03F202FA03F35B45C1
:1080200013D00494FFF727BB1D4B9C453FF702AECE
:10803000049B02932DE64FF4802501230BE4049A60
:1080400000F0BAF902460B4608E702F00102C2F15D
:1080500002020492FFF70FBB3E5555555555C53FDB
:1080600059F3F8C21F6EA501000000604715F73FE5
:1080700044DF5DF80BAE543E555555555555D53F2B
:10808000FE822B654715F73F9C7500883CE4377EE0
:108090000000F03FFFCB9040FEFFEF3F0000D03FDD
:1080A0000000E03FAFF3008021F0004C2DE9F843E1
:1080B0004FEA1C5CDFF86C814FEA0C5CC445064655
:1080C0000F460B46024600F08F8000296FDD0F152A
:1080D00078D0A7F2FF37C3F31303F90743F48013F3
:1080E00060D4D10F4FF0000C01EB43037F1052001E
:1080F000654616204FF400116C189C424FEAD27668
:108100004FEA420202DC1B1B65188C44013806EB67
:1081100043034FEA5101EFD1804620264FF0004142
:1081200009E023D0D40F013E4FEA510104EB430391
:108130004FEA42021ED0AB4201EB0804F1DD04F02D
:108140000049B9F1004F04EB010809D0A9465B1BB7
:10815000944288BF03F1FF33121B08444D46E1E708
:10816000B8F1000FF2DB05F10109F0E79442E6D91E
:108170001D46D7E71A4304D0431C41D000F0010349
:10818000184446084FEA6C031CF0010F03F17F53BB
:1081900003F5001318BF46F0004603EB07513046C5
:1081A000BDE8F883D10F01EB4303520099E721F0BA
:1081B0000043034322D051BB0F46D30A153F52055B
:1081C000002BFAD013F480111DD15B00D80201F10D
:1081D0000101FAD5C1F10100C1F1200422FA04F431
:1081E000234307448A4074E702460B4600F032FB03
:1081F00032463B4600F07CF9BDE8F883BDE8F883E1
:108200000CF1010CBEE7202401200021E6E7024624
:108210000B4600F06BF902460B4600F045FCBDE84A
:10822000F88300BF0000F07F21F00041704700BFDD
:1082300041F0004101F58010C00F704731F000435C
:1082400010B408D00F4AA3F5801494420AD8042031
:108250005DF8044B704700280CBF022003205DF836
:10826000044B7047B3F5801F01D20320F7E7064A9D
:10827000934201D00020F2E7D0F1010038BF002086
:10828000EDE700BFFFFFDF7F0000F07F00207047B9
:1082900000200149704700BF0000F87F2DE9F0433E
:1082A000C1F30A57A7F2FF36132E83B002460B46DE
:1082B000894684464FEAD17832DC002E4DDB3B49BB
:1082C000314101EA030010432FD0490801EA030CB1
:1082D0005CEA020C0DD04FF48029132E23EA010131
:1082E00049FA06F641EA060914BF4FF0000C4FF0B8
:1082F000004C2F4B03EBC8084F46D8E90089624673
:108300003B464046494600F0F3F8CDE900014246BD
:108310004B46DDE9000100F0E9F803B0BDE8F08369
:10832000332E07DDB6F5806F3DD01046194603B0F9
:10833000BDE8F083A7F213474FF0FF31F940014247
:10834000F3D049080142D4D04FF0804C20EA01011B
:108350004CFA07F741EA070CCBE721F00041014353
:10836000E3D0C3F31301124C0143484204EBC804A9
:10837000D4E900450843000B590C490400F40020DF
:1083800040EA01032046294600F0B2F8CDE9000199
:108390002B462246DDE9000100F0A8F821F0004359
:1083A00043EAC871C3E700F0A3F8C0E7FFFF0F007E
:1083B00030B60000FFFFFFFFC1F30A532DE9F04183
:1083C000904606460F460A461BBB21F00043034376
:1083D00034D03B4B002200F03DFA3A4B984506461C
:1083E0000F463BDBC1F30A53363B0A46434440F297
:1083F000FE718B4216DD32463B462DA1D1E90001CC
:1084000000F066F82AA3D3E9002300F023FABDE8C0
:10841000F08140F2FF74A34227D0434440F2FE7142
:108420008B42E8DC002B0BDD22F0FF4222F4E0025D
:1084300042EA035730463946BDE8F081BDE8F08195
:1084400013F1350F17DA4CF25033984532463B465C
:1084500020DC19A1D1E9000100F03AF816A3D3E914
:10846000002300F0F7F9BDE8F08102460B4600F06A
:108470003FF8BDE8F08122F0FF4222F4E0023633FB
:1084800042EA03573046394600220F4B00F0E2F92A
:10849000BDE8F08106A1D1E9000100F019F804A3BC
:1084A000D3E9002300F0D6F9BDE8F081AFF30080F6
:1084B0009C7500883CE4377E59F3F8C21F6EA50115
:1084C00000005043B03CFFFF0000903CAFF3008041
:1084D00030B403F0004321F0004243EA020130BC13
:1084E000704700BF81F0004102E000BF83F000430D
:1084F00030B54FEA41044FEA430594EA050F08BF3F
:1085000090EA020F1FBF54EA000C55EA020C7FEA02
:10851000645C7FEA655C00F0E2804FEA5454D4EB7F
:108520005555B8BF6D420CDD2C4480EA020281EA49
:10853000030382EA000083EA010180EA020281EA81
:108540000303362D88BF30BD11F0004F4FEA0131D3
:108550004FF4801C4CEA113102D0404261EB4101E2
:1085600013F0004F4FEA03334CEA133302D0524268
:1085700063EB430394EA050F00F0A780A4F1010424
:10858000D5F1200E0DDB02FA0EFC22FA05F280185E
:1085900041F1000103FA0EF2801843FA05F3594144
:1085A0000EE0A5F120050EF1200E012A03FA0EFCC3
:1085B00028BF4CF0020C43FA05F3C01851EBE371ED
:1085C00001F0004507D54FF0000EDCF1000C7EEB0A
:1085D00000006EEB0101B1F5801F1BD3B1F5001F48
:1085E0000CD349085FEA30004FEA3C0C04F1010467
:1085F0004FEA445212F5800F80F09A80BCF1004F90
:1086000008BF5FEA500C50F1000041EB045141EA11
:10861000050130BD5FEA4C0C404141EB010111F412
:10862000801FA4F10104E9D191F0000F04BF0146BD
:108630000020B1FA81F308BF2033A3F10B03B3F19B
:1086400020020CDA0C3208DD02F1140CC2F10C022B
:1086500001FA0CF021FA02F10CE002F11402D8BF89
:10866000C2F1200C01FA02F120FA0CFCDCBF41EA55
:108670000C019040E41AA2BF01EB0451294330BD24
:108680006FEA04041F3C1CDA0C340EDC04F1140401
:10869000C4F1200220FA04F001FA02F340EA0300D8
:1086A00021FA04F345EA030130BDC4F10C04C4F11E
:1086B000200220FA02F001FA04F340EA03002946FE
:1086C00030BD21FA04F0294630BD94F0000F83F448
:1086D000801306BF81F480110134013D4EE77FEA2B
:1086E000645C18BF7FEA655C29D094EA050F08BF77
:1086F00090EA020F05D054EA000C04BF1946104658
:1087000030BD91EA030F1EBF0021002030BD5FEA9B
:10871000545C05D14000494128BF41F0004130BDC3
:1087200014F580043CBF01F5801130BD01F0004517
:1087300045F0FE4141F470014FF0000030BD7FEA8A
:10874000645C1ABF194610467FEA655C1CBF0B4685
:10875000024650EA013406BF52EA033591EA030F9C
:1087600041F4002130BD00BF90F0000F04BF002194
:10877000704730B54FF4806404F132044FF00005C7
:108780004FF0000150E700BF90F0000F04BF002140
:10879000704730B54FF4806404F1320410F00045A6
:1087A00048BF40424FF000013EE700BF42004FEAA1
:1087B000E2014FEA31014FEA02701FBF12F07F431E
:1087C00093F07F4F81F06051704792F0000F14BF1B
:1087D00093F07F4F704730B54FF4607401F000455F
:1087E00021F0004120E700BF50EA010208BF7047B6
:1087F00030B54FF000050AE050EA010208BF7047AB
:1088000030B511F0004502D5404261EB41014FF413
:10881000806404F132045FEA915C3FF4DCAE4FF017
:1088200003025FEADC0C18BF03325FEADC0C18BFFE
:10883000033202EBDC02C2F1200300FA03FC20FA4F
:1088400002F001FA03FE40EA0E0021FA02F114449C
:10885000C1E600BF70B54FF0FF0C4CF4E06C1CEAB1
:1088600011541DBF1CEA135594EA0C0F95EA0C0F26
:1088700000F0DEF82C4481EA030621EA4C5123EA99
:108880004C5350EA013518BF52EA033541F48011C8
:1088900043F4801338D0A0FB02CE4FF00005E1FB7B
:1088A00002E506F00042E0FB03E54FF00006E1FBC5
:1088B00003569CF0000F18BF4EF0010EA4F1FF0408
:1088C000B6F5007F64F5407404D25FEA4E0E6D4148
:1088D00046EB060642EAC62141EA55514FEAC52059
:1088E00040EA5E504FEACE2EB4F1FD0C88BFBCF5D5
:1088F000E06F1ED8BEF1004F08BF5FEA500E50F186
:10890000000041EB045170BD06F0004646EA01014B
:1089100040EA020081EA0301B4EB5C04C2BFD4EB7D
:108920000C0541EA045170BD41F480114FF0000E76
:10893000013C00F3AB8014F1360FDEBF002001F0E4
:10894000004170BDC4F10004203C35DA0C341BDC5E
:1089500004F11404C4F1200500FA05F320FA04F030
:1089600001FA05F240EA020001F0004221F0004164
:1089700010EBD37021FA04F642EB06015EEA430ED7
:1089800008BF20EAD37070BDC4F10C04C4F1200507
:1089900000FA04F320FA05F001FA04F240EA0200BA
:1089A00001F0004110EBD37041F100015EEA430E8B
:1089B00008BF20EAD37070BDC4F1200500FA05F2AB
:1089C0004EEA020E20FA04F301FA05F243EA02032A
:1089D00021FA04F001F0004121FA04F220EA020039
:1089E00000EBD3705EEA430E08BF20EAD37070BD7F
:1089F00094F0000F0FD101F00046400041EB01015F
:108A000011F4801F08BF013CF7D041EA060195F040
:108A1000000F18BF704703F00046520043EB0303FA
:108A200013F4801F08BF013DF7D043EA06037047E7
:108A300094EA0C0F0CEA135518BF95EA0C0F0CD0F2
:108A400050EA410618BF52EA4306D1D181EA030138
:108A500001F000414FF0000070BD50EA410606BF32
:108A60001046194652EA430619D094EA0C0F02D177
:108A700050EA013613D195EA0C0F05D152EA0336BC
:108A80001CBF104619460AD181EA030101F00041DA
:108A900041F0FE4141F470014FF0000070BD41F023
:108AA000FE4141F4780170BD70B54FF0FF0C4CF4FD
:108AB000E06C1CEA11541DBF1CEA135594EA0C0F1C
:108AC00095EA0C0F00F0A7F8A4EB050481EA030E69
:108AD00052EA03354FEA013100F088804FEA033350
:108AE0004FF0805545EA131343EA12634FEA02221E
:108AF00045EA111545EA10654FEA00260EF00041DF
:108B00009D4208BF964244F1FD0404F5407402D230
:108B10005B084FEA3202B61A65EB03055B084FEAC1
:108B200032024FF480104FF4002CB6EB020E75EBBE
:108B3000030E22BFB61A754640EA0C005B084FEAE6
:108B40003202B6EB020E75EB030E22BFB61A754663
:108B500040EA5C005B084FEA3202B6EB020E75EBAE
:108B6000030E22BFB61A754640EA9C005B084FEA26
:108B70003202B6EB020E75EB030E22BFB61A754633
:108B800040EADC0055EA060E18D04FEA051545EA22
:108B900016754FEA06164FEAC30343EA52734FEACB
:108BA000C2025FEA1C1CC0D111F4801F0BD141EA44
:108BB00000014FF000004FF0004CB6E711F4801FA9
:108BC00004BF01430020B4F1FD0C88BFBCF5E06F89
:108BD0003FF6AFAEB5EB030C04BFB6EB020C5FEA99
:108BE000500C50F1000041EB045170BD0EF0004EEE
:108BF0004EEA113114EB5C04C2BFD4EB0C0541EA20
:108C0000045170BD41F480114FF0000E013C90E61C
:108C100045EA060E8DE60CEA135594EA0C0F08BFE0
:108C200095EA0C0F3FF43BAF94EA0C0F0AD150EADF
:108C300001347FF434AF95EA0C0F7FF425AF104672
:108C400019462CE795EA0C0F06D152EA03353FF49A
:108C5000FDAE1046194622E750EA410618BF52EA17
:108C600043067FF4C5AE50EA41047FF40DAF52EAEB
:108C700043057FF4EBAE12E74FF0FF3C06E000BF88
:108C80004FF0010C02E000BF4FF0010C4DF804CD95
:108C90004FEA410C7FEA6C5C4FEA430C18BF7FEA55
:108CA0006C5C1BD001B050EA410C0CBF52EA430C83
:108CB00091EA030F02BF90EA020F0020704710F103
:108CC000000F91EA030F58BF994208BF90422CBF92
:108CD000D8176FEAE37040F0010070474FEA410C8B
:108CE0007FEA6C5C02D150EA013C07D14FEA430CA9
:108CF0007FEA6C5CD6D152EA033CD3D05DF8040B1A
:108D0000704700BF8446104662468C46194663464B
:108D100000E000BF01B5FFF7B7FF002848BF10F122
:108D2000000F01BD4DF808EDFFF7F4FF0CBF012067
:108D300000205DF808FB00BF4DF808EDFFF7EAFFE3
:108D400034BF012000205DF808FB00BF4DF808ED9E
:108D5000FFF7E0FF94BF012000205DF808FB00BF93
:108D60004DF808EDFFF7CEFF94BF012000205DF81D
:108D700008FB00BF4DF808EDFFF7C4FF34BF01202A
:108D800000205DF808FB00BF4FEA410212F5001217
:108D900015D211D56FF47873B3EB625212D94FEA42
:108DA000C12343F0004343EA505311F0004F23FA2C
:108DB00002F018BF404270474FF00000704750EA81
:108DC000013005D111F0004008BF6FF0004070473E
:108DD0004FF00000704700BF80F0004002E000BF8D
:108DE00081F0004142001FBF5FEA410392EA030F96
:108DF0007FEA226C7FEA236C6AD04FEA1262D2EBE0
:108E00001363C1BFD218414048404140B8BF5B42E4
:108E1000192B88BF704710F0004F40F4000020F07D
:108E20007F4018BF404211F0004F41F4000121F093
:108E30007F4118BF494292EA030F3FD0A2F10102DD
:108E400041FA03FC10EB0C00C3F1200301FA03F11B
:108E500000F0004302D5494260EB4000B0F5000F3E
:108E600013D3B0F1807F06D340084FEA310102F1FD
:108E70000102FE2A51D2B1F1004F40EBC25008BFAF
:108E800020F0010040EA03007047490040EB000079
:108E900010F4000FA2F10102EDD1B0FA80FCACF1A8
:108EA000080CB2EB0C0200FA0CF0AABF00EBC250A7
:108EB00052421843BCBFD0401843704792F0000F95
:108EC00081F4000106BF80F400000132013BB5E7E8
:108ED0004FEA41037FEA226C18BF7FEA236C21D05E
:108EE00092EA030F04D092F0000F08BF08467047C3
:108EF00090EA010F1CBF0020704712F07F4F04D191
:108F0000400028BF40F00040704712F100723CBFA3
:108F100000F50000704700F0004343F0FE4040F4CD
:108F2000000070477FEA226216BF08467FEA23638B
:108F30000146420206BF5FEA412390EA010F40F476
:108F4000800070474FF0000304E000BF10F00043C2
:108F500048BF40425FEA000C08BF704743F09643A9
:108F600001464FF000001CE050EA010208BF7047C4
:108F70004FF000030AE000BF50EA010208BF70474B
:108F800011F0004302D5404261EB41015FEA010C60
:108F900002BF84460146002043F0B64308BFA3F158
:108FA0008053A3F50003BCFA8CF2083AA3EBC2533A
:108FB00010DB01FA02FC634400FA02FCC2F1200259
:108FC000BCF1004F20FA02F243EB020008BF20F090
:108FD0000100704702F1200201FA02FCC2F12002F6
:108FE00050EA4C0021FA02F243EB020008BF20EAEB
:108FF000DC7070474FF0FF0C1CEAD0521EBF1CEA19
:10900000D15392EA0C0F93EA0C0F6FD01A4480EA06
:10901000010C400218BF5FEA41211ED04FF00063EF
:1090200043EA501043EA5111A0FB01310CF000401B
:10903000B1F5000F3EBF490041EAD3715B0040EA41
:10904000010062F17F02FD2A1DD8B3F1004F40EB11
:10905000C25008BF20F00100704790F0000F0CF0E4
:10906000004C08BF49024CEA502040EA51207F3AA8
:10907000C2BFD2F1FF0340EAC250704740F4000083
:109080004FF00003013A5DDC12F1190FDCBF00F074
:1090900000407047C2F10002410021FA02F1C2F122
:1090A000200200FA02FC5FEA310040F1000053EABE
:1090B0004C0308BF20EADC70704792F0000F00F00C
:1090C000004C02BF400010F4000F013AF9D040EA12
:1090D0000C0093F0000F01F0004C02BF490011F4A6
:1090E000000F013BF9D041EA0C018FE70CEAD153A4
:1090F00092EA0C0F18BF93EA0C0F0AD030F0004C24
:1091000018BF31F0004CD8D180EA010000F00040D7
:10911000704790F0000F17BF90F0004F084691F095
:10912000000F91F0004F14D092EA0C0F01D14202CF
:109130000FD193EA0C0F03D14B0218BF084608D198
:1091400080EA010000F0004040F0FE4040F40000E2
:10915000704740F0FE4040F4400070474FF0FF0C75
:109160001CEAD0521EBF1CEAD15392EA0C0F93EABC
:109170000C0F69D0A2EB030280EA010C49024FEA0E
:10918000402037D04FF0805343EA111143EA1013C7
:109190000CF000408B4238BF5B0042F17D024FF47F
:1091A000000C8B4224BF5B1A40EA0C00B3EB510F5A
:1091B00024BFA3EB510340EA5C00B3EB910F24BF43
:1091C000A3EB910340EA9C00B3EBD10F24BFA3EBC8
:1091D000D10340EADC001B0118BF5FEA1C1CE0D190
:1091E000FD2A3FF650AF8B4240EBC25008BF20F043
:1091F000010070470CF0004C4CEA50207F32C2BF97
:10920000D2F1FF0340EAC250704740F400004FF033
:109210000003013A37E792F0000F00F0004C02BF64
:10922000400010F4000F013AF9D040EA0C0093F02E
:10923000000F01F0004C02BF490011F4000F013B88
:10924000F9D041EA0C0195E70CEAD15392EA0C0FF0
:1092500008D142027FF47DAF93EA0C0F7FF470AF28
:10926000084676E793EA0C0F04D14B023FF44CAF6B
:1092700008466EE730F0004C18BF31F0004CCAD100
:1092800030F000427FF45CAF31F000437FF43CAF3C
:109290005FE700BF4FF0FF3C06E000BF4FF0010C5E
:1092A00002E000BF4FF0010C4DF804CD4FEA400240
:1092B0004FEA41037FEA226C18BF7FEA236C11D08A
:1092C00001B052EA530C18BF90EA010F58BFB2EB3D
:1092D000030088BFC81738BF6FEAE17018BF40F0BD
:1092E000010070477FEA226C02D15FEA402C05D171
:1092F0007FEA236CE4D15FEA412CE1D05DF8040BF6
:10930000704700BF844608466146FFE70FB5FFF788
:10931000C9FF002848BF10F1000F0FBD4DF808ED40
:10932000FFF7F4FF0CBF012000205DF808FB00BF31
:109330004DF808EDFFF7EAFF34BF012000205DF88B
:1093400008FB00BF4DF808EDFFF7E0FF94BF0120D8
:1093500000205DF808FB00BF4DF808EDFFF7D2FFD5
:1093600094BF012000205DF808FB00BF4DF808ED18
:10937000FFF7C8FF34BF012000205DF808FB00BFE5
:109380004FEA4002B2F1FE4F0FD34FF09E03B3EB12
:1093900012620DD94FEA002343F0004310F0004F52
:1093A00023FA02F018BF404270474FF000007047A8
:1093B00012F1610F01D1420205D110F0004008BF47
:1093C0006FF0004070474FF00000704703460846BA
:1093D000194600F005B800BF00210A2201F0A0BB29
:1093E00010B40C4613460146224602205DF8044B99
:1093F00001F0A2BB014B1868704700BF7894FF1FB3
:1094000070B50F4E0F4D761BB61007D0043D0024EB
:10941000013455F8043F9847A642F9D10A4E0B4D46
:10942000761B02F093F9B61008D0043D00240134F5
:1094300055F8043F9847A642F9D170BD70BD00BFF2
:1094400058B7000058B7000098B7000058B70000A0
:10945000024B0146186800F00BB800BF7894FF1F5C
:10946000024B0146186801F031BC00BF7894FF1F21
:109470002DE9F04F01F10B05162D83B0064627D9D3
:1094800035F0070527D4A94225D8304600F06AFBFD
:10949000B5F5FC7F26D2C14F4FEAD50C07EBCC03C4
:1094A000DC689C4200F0D2816368E268A16823F026
:1094B0000303234430465D68CA6045F001059160AE
:1094C0005D6000F051FB0834204603B0BDE8F08F2A
:1094D0001025A942D9D900240C232046336003B0BB
:1094E000BDE8F08F5FEA552C00F08A80BCF1040FD4
:1094F00000F260814FEA951C0CF1380C4FEA4C01E8
:10950000A64F07EB8101CC68A14205D10CE0002BEE
:109510007ADAE468A14207D0626822F00302531BA2
:109520000F2BF4DD0CF1FF3C0CF1010C9B4B3C6963
:1095300003F1080E744500F07E81616821F003019B
:109540004A1B0F2A00F36481002AC3F814E0C3F811
:1095500010E06ADAB1F5007F80F03A81C90803EBC8
:10956000C1004FEAA1085A688168A1604FF0010963
:1095700009FA08F848EA0202E0605A608460CC60A8
:109580004FEAAC030120984090425BD8024206D1DA
:109590002CF0030C400002420CF1040CFAD007EB53
:1095A000CC084446E146E3689C4207D145E1002AE5
:1095B00080F25681DB689C4200F03F81596821F0BF
:1095C00003014A1B0F2AF2DD1C46D3F80CC054F8E5
:1095D000088F591945F0010942F00105C3F80490BC
:1095E0003046C8F80CC0CCF8088079613961C1F800
:1095F0000CE0C1F808E04D608A5000F0B5FA63E76E
:109600007E214FF03F0C7BE72244E3685068A1685D
:1096100040F00105CB6030469960556000F0A4FA37
:109620000834204603B0BDE8F08F214430464B6833
:1096300043F001034B6000F097FA0834204603B072
:10964000BDE8F08FBC68636823F00309A94504D323
:10965000C5EB09030F2B00F39180514B514A196858
:109660001368013305EB010A04EB090B00F061817B
:109670000AF5805A0AF10F0A2AF47F6A2AF00F0AC3
:1096800030465146019200F00DFFB0F1FF3F804699
:10969000019A00F00081834500F2FA80DFF810C1E2
:1096A000DCF80030C3455344CCF8003000F04A8168
:1096B00012683C4901321BBFCBEB080B5B44C1F87D
:1096C0000080CCF8003018F0070300F01381C3F1DC
:1096D0000802C3F5805390440833C244CAF30B0A0E
:1096E000CAEB030A51463046CDF804C000F0DAFE5A
:1096F000431CDDF804C000F03581C8EB0002524481
:1097000042F00102DCF80030C7F808805344BC4244
:10971000C8F80420CCF80030DFF894A015D0B9F1D7
:109720000F0F40F2EA806168A9F10C0222F00702F3
:1097300001F0010EA118052042EA0E0E0F2AC4F80E
:1097400004E04860886000F21181174ABC68116823
:109750008B4288BF1360154A11688B4288BF136023
:10976000626822F003029542C5EB020301D80F2B79
:1097700004DC304600F0F8F90024A5E6621943F055
:10978000010345F0010565603046BA60536000F0A2
:10979000EBF90834204603B0BDE8F08F7C94FF1F3E
:1097A00050FFFF1F8898FF1F4CFFFF1F48FFFF1F40
:1097B00054FFFF1FBCF1140F61D9BCF1540F00F22C
:1097C0008F804FEA153C0CF16E0C4FEA4C0197E686
:1097D0004B0A042B58D9142B00F2AE8003F15B0224
:1097E000500007EB8000DFF8BC818368834200F003
:1097F0008A805A6822F00302914202D29B68984202
:10980000F7D1D9687A68E160A3608C60DC60B7E664
:10981000611942F0010745F0010565603046596164
:109820001961C1F80CE0C1F808E04F608A500834B3
:1098300000F09AF948E65A68A2E609F1010919F020
:10984000030F04F108047FF4AEAE2DE004F1080329
:109850006469A34208BF0CF1020C3FF467AE23E633
:1098600019441C464868DB6854F8082F40F001058D
:109870004D603046D3609A6000F076F924E60CF132
:109880005B0C4FEA4C013BE68A0938325000A8E7EE
:10989000BC423FF403AFBC68626822F0030262E797
:1098A000D8F8008098457BD11CF0030FA8F108037D
:1098B0000CF1FF3CF4D17B6823EA00037B6040009D
:1098C00098423FF6BFAE00283FF4BCAE0342CC4600
:1098D0007FF465AE400003420CF1040CFAD05EE662
:1098E000BCF5AA7F1AD84FEAD53C0CF1770C4FEAA9
:1098F0004C0105E64FF48053EFE60123C8F804302D
:10990000444600222FE791100120D8F8042000FAE5
:1099100001F10A43C8F80420194674E740F2545391
:109920009C451BD84FEA954C0CF17C0C4FEA4C013E
:10993000E6E50AF1100AA3E6542B1FD80A0B6E3293
:1099400050004EE7CBF30B0100297FF4B1AE0AEBD8
:109950000901BA6841F001015160F6E6FC214FF0BF
:109960007E0CCDE501224FF0000ACBE604F10801A0
:10997000304601F0ABF9DAF80030E6E6B3F5AA7F3D
:1099800003D8CA0B773250002BE740F2545293426F
:1099900003D88A0C7C32500023E7FC207E2220E78B
:1099A0007B688CE77C94FF1F032A70B428D940EAB7
:1099B00001039B0713D005780C78A54224D1013A06
:1099C000002305E010F8015F11F8014FA5421BD1FB
:1099D000934203F10103F5D1002070BC70470C469F
:1099E000034625681E68AE422146184604F1040469
:1099F00003F1040304D1043A032A18462146F0D89F
:109A0000002AD8D11046E8E7281B70BC704700BF79
:109A10008842F0B410D98C18A0420DD28518531E7C
:109A200042B121462A4611F8014D02F8014D013B91
:109A30005C1CF8D1F0BC70470F2A3FD940EA010303
:109A40009B073FD1A2F110073F0900EB0716103624
:109A50000C46034625681D6065685D60A5689D60CD
:109A6000E568DD601033B34204F11004F2D17B1CD1
:109A700002F00F0C1B01BCF1030F1944034423D95E
:109A80000E461D466446043C56F8047B45F8047BAC
:109A9000032CF8D8ACF1040424F00304043402F0DD
:109AA000030223442144002AC4D01A4411F8014B74
:109AB00003F8014B9342F9D1F0BC70470346002AEA
:109AC000F3D1B7E70346F0E76246002AEDD1B1E7EC
:109AD000F0B4840743D0541E002A3ED0CDB20346D2
:109AE00003E0621E002C38D0144603F8015B9A078D
:109AF000F7D1032C2AD9CDB245EA05250F2C45EA2A
:109B0000054515D9A4F110073F0903F1100606EB2E
:109B100007161A46156055609560D5601032B2423E
:109B2000F8D104F00F040137032C03EB07130DD910
:109B30001E462246043A032A46F8045BFAD8221F3E
:109B400022F003020432134404F003042CB1C9B21E
:109B50001C4403F8011BA342FBD1F0BC7047144620
:109B60000346C6E7704700BF704700BF2DE9F04FBE
:109B700087B0044600920098019102EB4202520025
:109B800005928008A2071D46029040F0838000994C
:109B90008B077FD1019AB1F1040918BF4FF0010979
:109BA000062A7CD9019A00985308072A00FB034B28
:109BB00040F00281059E2644B9F1000F40F01B8160
:109BC0002168DBF800202260CBF80010009B009891
:109BD00023444FF0000AD34604931F460393C0F179
:109BE0000008B246B74240F296805346DA469B469A
:109BF000BAF1000F00F0D381039A9DE80900B91A69
:109C0000C4EB020C8C45A8BF8C4600FB0343BCF19F
:109C1000000F019311DDB9F1020FCCEB070040F00A
:109C2000448104EB0C0A224690F800C0137802F835
:109C300001CB524500F8013BF6D1019B0098CBEBDC
:109C40000302C6EB0B06121AB24228BF3246002AA4
:109C500010DD0198B9F1020FC2EB000340F0428120
:109C600007EB020C18783A7807F8010B674503F800
:109C7000012BF7D1009A8A42C0F0CE80009CB442FA
:109C800046D201980099841BA207B6FBF1F6019613
:109C90003FF47DAF019A062A4FF0020982D8009B5B
:109CA000984603FB024BA044D84531D25F42DDF811
:109CB00000A0CDF804B023464C469946C14523D2B6
:109CC000464608E03268DBF800303360CBF800200D
:109CD000CB4519D95E4606EB070B58463146A847D7
:109CE000002811DD002CEDD0012C00F0A18152469E
:109CF0005B46013A3178187806F8010B002A03F820
:109D0000011BF6DCCB45E5D8019AD0449045D5D36C
:109D100007B0BDE8F08F38462146A84700280DDC83
:109D200036E03268DAF800303360CAF80020C24406
:109D30004FF0010B4644B7423FF657AF304621463D
:109D4000A8470028C0F29081F4D1B9F1000FE8D003
:109D5000B9F1010F0DD000995246334601391878F8
:109D600092F800C003F801CB002902F8010BF5DCE2
:109D7000DDE7029B50463146A446013B0C68026871
:109D800041F8042B002B40F8044BF6DC6446CEE788
:109D90000FD1B9F1000F40F0B280039B03981A680D
:109DA0003B6803603A60039A009B1A4403924FF0A9
:109DB000010B0098074415E7019A009B561E282ABC
:109DC00003FB064631D8B046274659463846A847D1
:109DD00000284146584679DBA84700283FF7ECAEFB
:109DE00038464146A84738EA200B28BFBB46B9F1A0
:109DF000000F3FF4E5AEB9F1010F00F09180009A39
:109E000059462346013A18780F7803F8017B002A57
:109E100001F8010BF6DCD9E62046009C2B46B1FB8D
:109E2000F4F12246FFF7A2FE28E74FEAD20803FB2F
:109E300008F804EB08074FEA4802394620469246E4
:109E40000392A847A244002851463846C0F29B809E
:109E5000A847002840F30081C8F100039A46DA447D
:109E6000594650460493A847D844002841465846CE
:109E70007EDBA847002840F3E780039ADDF81080D6
:109E8000C2EB060AB04441465046A8470028314676
:109E9000404652DBA847002897DC50463146A84789
:109EA00036EA200828BFD0468FE74FEA9C0C2246AE
:109EB00088460CF1FF3C1168036842F8043BBCF192
:109EC000000F40F8041BF4DC4146B6E6A847002822
:109ED000FFF672AE38464146A84737EA200B28BF46
:109EE000C34669E692088C46013A3968186847F813
:109EF000040B002A43F8041BF6DC6146BAE6B9F10C
:109F0000010F26D00099039B3A460139187892F840
:109F100000C003F801CB002902F8010BF5DC42E791
:109F2000029A5B462146013A0F68186841F8040B13
:109F3000002A43F8047BF6DC48E6A8470028FFF631
:109F400044AF50463146A8473AEA200828BFB046F9
:109F50003BE70399029B3846A446013B0C68026824
:109F600041F8042B002B40F8044BF6DC64461AE75A
:109F7000A847002881DB50464146A8473AEA200B13
:109F800028BFC34679E7A8470028FFF665AF2046FB
:109F90005146A84734EA200728BF57465CE7019A94
:109FA000009B03FB0248049A4245BFF4B1AE5F42F6
:109FB000DDF800B0CDF80480234692464C46994621
:109FC000D14522D2564608E03268D8F800303360D6
:109FD000C8F80020C84518D9464606EB0708404691
:109FE0003146A847002810DD002CEDD0012C13D0FD
:109FF0005A464346013A3178187806F8010B002A90
:10A0000003F8011BF6DCC845E6D8019BDA449A4503
:10A01000D6D307B0BDE8F08F029B4146013B3068C4
:10A020000A6846F8042B002B41F8040BF6DCD1E754
:10A03000029B5946013B30680A6846F8042B002B06
:10A0400041F8040BF6DC43E650464146A84738EA9F
:10A05000200B28BFD34610E720465146A8473AEACE
:10A06000200728BF2746F7E6B7423FF6BEADB9F155
:10A07000000F09D13A6833683B60326000994FF0B5
:10A08000010B0F44761AADE5B9F1010F0DD000991F
:10A0900032463B460139187892F800C003F801CBEC
:10A0A000002902F8010BF5DCE8E7029B304639464F
:10A0B000A446013B0C68026841F8042B002B40F8D1
:10A0C000044BF6DC6446D9E7024B0A4601461868A1
:10A0D00000F002B87894FF1F2DE9F04F0C4683B0D2
:10A0E00090468146002900F0E280FFF73BFD08F131
:10A0F0000B0654F8043C162E23F00305A4F10807C0
:10A100004BD810210E46B0454CD88D4278DADFF896
:10A1100090B3DBF808E07819864500F0CE804268FD
:10A1200022F0010C8444DCF804C01CF0010F7AD04A
:10A1300000221046DB0700F1928054F8083CC3EB84
:10A14000070ADAF8043023F003032B4488B3704580
:10A1500000F0ED8002EB030E8E452ADBC3688268B7
:10A160005746D3609A6057F8081FDAF80C30CB6076
:10A170002A1F242A996000F22681132A40F2B38014
:10A180002368CAF808306368CAF80C301B2A00F24A
:10A19000308108340AF11003A6E026F00706002EED
:10A1A0003146B0DA0C230020C9F8003003B0BDE816
:10A1B000F08F8B4253DB5746DAF80C1057F8080F34
:10A1C0002A1F242AC160886000F20981132A40F204
:10A1D00004812168CAF808106168CAF80C101B2AAB
:10A1E00000F21C8108340AF11002216811606168D4
:10A1F0005160A16891601D46DAF804303C4657462C
:10A20000AA1B0F2A03F0010319D82B433D447B609E
:10A210006B6843F001036B604846FFF7A5FC2046DE
:10A2200003B0BDE8F08F22F0030202EB050C8C4571
:10A2300080DBC26881686546CA609160E0E7B91951
:10A2400042F001001E430A447E604860536843F0B8
:10A25000010308315360484600F038FDDCE7414611
:10A260004846FFF705F98046D0B154F8043C23F086
:10A2700001023A44A0F10801914200F09E802A1F99
:10A28000242A50D8132A23D803462246116819607D
:10A290005168596092689A602146484600F016FD60
:10A2A0004846FFF761FC404603B0BDE8F08F114619
:10A2B00003B0BDE8F04FFFF7DBB8DEF8042022F072
:10A2C0000302501906F1100C604519DA704631E7A7
:10A2D00023680360636843601B2A63D800F10803A6
:10A2E00004F10802D2E73B4622681A6062685A60AD
:10A2F000A2689A603C467546DAF8043057467FE714
:10A300003744831B43F00103CBF808707B6054F89B
:10A31000043C03F001031E43484644F8046CFFF775
:10A3200023FC20467CE72146FFF772FBB4E702EBF3
:10A33000030C06F110029445FFF63BAF5746DAF8DE
:10A340000C3057F8081F2A1F242ACB60996000F2AE
:10A350008780132A78D92368CAF808306368CAF856
:10A360000C301B2A00F2858008340AF110032268A1
:10A370001A6062685A60A2689A600AEB0603C6EB2C
:10A380000C0242F00102CBF808305A60DAF80430CF
:10A3900003F001031E434846CAF80460FFF7E4FBDC
:10A3A00038463DE7A3688360E368C360242A2CD065
:10A3B00000F1100304F1100268E750F8042C22F0B9
:10A3C000030215441CE72146384675463C46FFF714
:10A3D0001FFB5746DAF8043012E73A4605E72146F4
:10A3E00038461D463C46FFF713FB5746DAF8043063
:10A3F00006E7A368CAF81030E368CAF81430242AC4
:10A4000018D010340AF118036EE7236903616369F9
:10A41000436104F1180200F1180337E7A168CAF894
:10A420001010E168CAF81410242A0FD010340AF171
:10A430001802DAE62369CAF818306369CAF81C30D2
:10A4400018340AF120034FE73B4690E72269CAF827
:10A4500018206269CAF81C2018340AF12002C4E6E8
:10A4600021463846CDF804C0FFF7D2FADDF804C023
:10A4700083E7A368CAF81030E368CAF81430242AC6
:10A4800003D010340AF1180371E72369CAF81830B1
:10A490006369CAF81C3018340AF1200367E700BF6B
:10A4A0007C94FF1F38B5074C0023054608462360FF
:10A4B000F9F762FF431C00D038BD2368002BFBD0A6
:10A4C0002B6038BD90FFFF1FC9B2F0B4002947D000
:10A4D00085070FD00278002A3FD091423ED0431C1E
:10A4E00005E013F8012B002A37D0914236D09A07A5
:10A4F0001846F6D1036841EA012747EA074783EA8D
:10A500000702A2F10135A3F1013425EA020224EA8F
:10A510000303134313F0803F11D1021D104652F87C
:10A52000043B83EA0704A4F10136A3F1013526EACE
:10A53000040425EA0303234313F0803FEED003789D
:10A54000002B39D0994209D0431C01E0914205D03B
:10A55000184613F8012B002AF8D11046F0BC7047BA
:10A5600084070BD00378002BF8D0431C03E002785B
:10A570000133002AF2D099071846F8D10368A3F1F5
:10A58000013222EA030313F0803F0AD1031D18466B
:10A5900053F8042BA2F1013121EA020212F0803FAC
:10A5A000F5D00378002BD9D0431C1846013302782C
:10A5B000002AFAD1F0BC70471846CFE740EA010CF8
:10A5C0001CF0070F23D1BDF1100DCDE90245CDE9F7
:10A5D00000676FF000064FF0000700BFF0E80223AD
:10A5E000F1E80245A24282FA46FCA7FA86FC08BFBF
:10A5F000BCF1000F40F0D780AB4283FA46FCA7FACB
:10A6000086FC08BFBCF1000F40F0CA80E6E710F0FE
:10A61000030C21D020F0030050F8042B5FEACC7C1F
:10A6200008D00FD211F801CB5FFA92F3B3EB0C0C08
:10A6300010D17BB111F801CB5FFAA2F3B3EB0C0C94
:10A6400008D13BB111F801CB5FFAB2F3B3EB0C0CBC
:10A6500000D10BB960467047BDF1100DCDE9024540
:10A66000CDE900676FF000064FF0000711F0030C12
:10A670002DD110F0040F0DD050F8042B51F8044BDD
:10A68000A24282FA46FCA7FA86FC08BFBCF1000F82
:10A6900040F0898011F0040F9FD051F8045B00BF97
:10A6A000F0E80223AA4282FA46FCA7FA86FC08BF19
:10A6B000BCF1000F71D1F1E80245A34283FA46FCD8
:10A6C000A7FA86FC08BFBCF1000F63D1E8E721F0D0
:10A6D0000301BCF1020F1ED03BDA51F8045B00BF4E
:10A6E00050F8043B4FEA152583FA46FCA7FA86FC8E
:10A6F000B7EB0C2F03EA162208BFAA424DD151F83E
:10A70000045BBCF1000F82EA03034FEA056208BF55
:10A7100093423CD1E4E751F8045B00BF50F8043B9E
:10A720004FEA154583FA46FCA7FA86FCB7EB0C4FB7
:10A7300003EA164208BFAA422FD151F8045BBCF1CC
:10A74000000F82EA03034FEA054208BF93421ED17D
:10A75000E4E751F8045B00BF50F8043B4FEA15658D
:10A7600083FA46FCA7FA86FCB7EB0C6F03EA166285
:10A7700008BFAA4211D151F8045BBCF1000F82EA74
:10A7800003034FEA052208BF934200D1E4E719BA58
:10A7900012BA0AE019BA22BA07E011BA2ABA04E0DA
:10A7A00019BA2ABA01E011BA22BA9CFA8CF0DDE992
:10A7B0000067DDE902451DF1100D38B1B0FA80F0F7
:10A7C000C0F1180021FA00F122FA00F201209142B2
:10A7D00098BF8041704700BF80EA0102844612F0B2
:10A7E000030F4FD111F0030F32D14DF8044D11F08A
:10A7F000040F51F8043B0BD0A3F101329A4312F03D
:10A80000803F04BF4CF8043B51F8043B16D100BF15
:10A8100051F8044BA3F101329A4312F0803FA4F1A6
:10A8200001320BD14CF8043BA24312F0803F04BF2D
:10A8300051F8043B4CF8044BEAD023460CF8013B9A
:10A8400013F0FF0F4FEA3323F8D15DF8044B704744
:10A8500011F0010F06D011F8012B0CF8012B002A82
:10A8600008BF704711F0020FBFD031F8022B12F071
:10A87000FF0F16BF2CF8022B8CF8002012F47F4F2C
:10A88000B3D1704711F8012B0CF8012B002AF9D134
:10A89000704700BF20F0030110F00300C0F100007A
:10A8A00051F8043B00F1040C4FEACC0C6FF00002AD
:10A8B0001CBF22FA0CF213434FF0010C4CEA0C2C93
:10A8C0004CEA0C4CA3EB0C0222EA030212EACC1273
:10A8D00004BF51F8043B0430F4D013F0FF0F1FBF46
:10A8E000013013F47F4F013013F47F0F18BF013094
:10A8F000704700BF30B4002A4AD040EA010313F089
:10A9000003032DD1032A2BD904680D68AC4227D14B
:10A91000043A3DD0A4F1013525EA040414F0803F47
:10A920003CD10C4603460EE05B686468A3F1013538
:10A93000A34225EA030513D1043A29D015F0803F3C
:10A9400029D103460C46032A00F1040001F1040159
:10A95000EAD8551E2AB918792279801A30BC704776
:10A96000551E03780A7893421AD1DDB1B3B16C1C3D
:10A970000C448B1C014604E0A3420CD00133002898
:10A98000ECD011F8010F13F8012C9042F4D0E4E759
:10A99000104630BC7047002030BC70471846DDE7D9
:10A9A0001846DAE72846D9E740EA01039B0770B466
:10A9B0002AD1032A28D90C460346214654F8045BC1
:10A9C000A5F1013626EA050616F0803F05D1043AC6
:10A9D000032A43F8045B2146EFD89AB10C781C7027
:10A9E000013A01333CB16AB111F8014F03F8014B50
:10A9F000013A002CF7D12AB11A44002103F8011BB7
:10AA00009342FBD170BC70470346E6E72DE9F00F97
:10AA1000424C82B0D4F800C001900E4600E02646B9
:10AA2000344614F8015B0CEB0500407800F0080098
:10AA300000F0FF0A0028F2D12D2D5BD02B2D04BF92
:10AA40007578B41C33F010003CD09946BAF1000F71
:10AA50000CBF6FF0004B4FF0004BBBFBF9F8002729
:10AA600009FB18BB38460CE0303DAB4219DD7E1CBB
:10AA700005D0404523D820D009FB0050012714F809
:10AA8000015B0CEB0506767816F0040FECD116F09E
:10AA9000030606D0012E14BF57263726AD1BAB4246
:10AAA000E5DC7B1C15D0BAF1000F21D10AB1EFB95A
:10AAB000116002B0BDE8F00F70475D45DCDD4FF07E
:10AAC000FF37DCE7302D1AD0002BBED10A23994680
:10AAD000BCE70199BAF1000F4FF022030CBF6FF0F1
:10AAE00000404FF000400B60002AE2D0611EDFE71B
:10AAF0004042DBE7B41C75784FF0010AA2E72078EA
:10AB000000F0DF00582803D0002B9ED108239CE7DB
:10AB1000102365789946023498E700BF8C98FF1F90
:10AB200030B4044C0D46134601462A46206830BC1A
:10AB3000FFF76CBF7894FF1FF0B5274C2668D6F856
:10AB4000484185B00746002C41D065681F2D1EDDA9
:10AB5000224818B94FF0FF3005B0F0BD4FF4C8706F
:10AB6000039102920193FEF773FC0399029A019BF1
:10AB700004460028EED0D6F84851256000206060D9
:10AB80000546C6F84841C4F88801C4F88C013FB9AD
:10AB9000AB1C00200135656044F8231005B0F0BD02
:10ABA00004EB85004FF0010CC0F88820D4F88861D0
:10ABB0000CFA05F21643022FC4F88861C0F8083178
:10ABC000E6D1D4F88C311A43C4F88C21E0E706F5BD
:10ABD000A674C6F84841B8E744B600005194000096
:10ABE000024B13B1024800F005B8704700000000A6
:10ABF00001AC00000146002002460346FFF79CBF5F
:10AC000038B5094D094C641BA41018BF05EB840529
:10AC100005D0013C55F8043D9847002CF9D1BDE81A
:10AC2000384000F0B9BD00BF000000000000000087
:10AC3000F8B5234D0F460446FEF794FFAB685E68F7
:10AC400026F00306F11B01F6EF7121F47F6121F07C
:10AC50000F01A1F58057B7F5805F07DB2046002183
:10AC6000FFF720FCAB683344984204D02046FEF73F
:10AC70007BFF0020F8BD20467942FFF713FC01302E
:10AC80000DD0104BAA681968F61B46F00106204645
:10AC9000C91B56601960FEF767FF0120F8BD20460A
:10ACA0000021FFF7FFFBAB68C21A0F2ADEDD064D5D
:10ACB00004492D6842F00102401B5A600860D5E744
:10ACC0007C94FF1F54FFFF1F8898FF1F2DE9F04160
:10ACD0000D460646002955D0FEF744FF55F8041CE2
:10ACE000DFF874C121F00103A5F10804E218DCF8D3
:10ACF00008005768904227F0030769D011F001015E
:10AD0000576032D00021D0194068C00706D43B44B8
:10AD1000906800294ED0D268C260906043F0010272
:10AD20006260E350E1B9B3F5007F2DD35A0A042ADB
:10AD30006AD89809383041000CEB810C4649DCF8A0
:10AD40000820624566D0516821F003018B4202D28F
:10AD500092689445F7D1D368E360A2609C60D460A8
:10AD60003046BDE8F041FEF7FFBE55F8085C641BB5
:10AD70000CF10808A06840452B4443D0E568C56045
:10AD8000A860C0E7BDE8F081DB080CEBC302012539
:10AD9000DCF804009168A1609B1005FA03F31843E6
:10ADA000E260CCF8040094603046CC60BDE8F0412D
:10ADB000FEF7DABE294DA842ADD143F00102CCF82E
:10ADC0001440CCF81040E060A0606260E350C7E738
:10ADD0001F44CB0707D455F8083CE41A1F44A26867
:10ADE000E368D3609A601E4B1B6847F001029F42E4
:10ADF0006260CCF80840B3D31A4B30461968FFF7AD
:10AE000017FFADE701217EE7142A0CD802F15B00A1
:10AE1000410091E74B688010012505FA00F00343DB
:10AE20004B60134698E7542A03D8180B6E30410044
:10AE300082E7B2F5AA7F03D8D80B773041007BE7D1
:10AE400040F254518A4203D8980C7C30410073E799
:10AE5000FC217E2070E700BF7C94FF1F8494FF1FBD
:10AE60008498FF1F50FFFF1F00000000000000003B
:10AE70008943000000000000486F74737761702000
:10AE800063616C6C656400005F00000053504F54B8
:10AE90004C00000054524153480000002F000000B5
:10AEA0007C00000042616E6B3A0000002043686144
:10AEB0006E6E656C3A0000002046696C653A0000D1
:10AEC00042616E6B3A200000200000002046696C51
:10AED000657320666F756E64000000002920000015
:10AEE000207C20004D5554453D0000004445434C16
:10AEF00049434B3D0000000053686F774D65746512
:10AF0000723D00006D65746572484944453D00001E
:10AF10004368616E506F74496D6D656469617465F5
:10AF20003D0000004368616E4356496D6D6564697C
:10AF30006174653D000000005374617274506F7459
:10AF4000496D6D6564696174653D0000537461729B
:10AF5000744356496D6D6564696174653D00000018
:10AF60004D555445000000004445434C49434B00B7
:10AF700053686F774D657465720000006D65746588
:10AF800072484944450000004368616E506F74493F
:10AF90006D6D656469617465000000004368616EF1
:10AFA0004356496D6D6564696174650053746172DF
:10AFB00074506F74496D6D6564696174650000005B
:10AFC00053746172744356496D6D6564696174654B
:10AFD00000000000537461727443564469766964DA
:10AFE000657200004C6F6F70696E6700536F72740A
:10AFF0000000000073657474696E67732E74787452
:10B00000000000006572726F72206F70656E696E6D
:10B01000672073657474696E67732E7478740000AA
:10B0200053746172744356446976696465723D0075
:10B030004C6F6F70696E673D00000000536F727453
:10B040003D000000467265652072616D3A20000087
:10B05000506C6179686561643A2000005241570084
:10B060003000FFFF0000010004000B0013001E0071
:10B070002C003C004E0063007B009500B100D00026
:10B08000F10014013A0163018E01BB01EA011D02C6
:10B0900051028802C102FC023A037B03BD03020491
:10B0A00049049304DF042D057D05D00524067C06A4
:10B0B000D50630078E07EE075008B4081A09830931
:10B0C000ED095A0AC90A390BAC0B210C980C100D6A
:10B0D0008B0D080E860E070F890F0D1093101B1194
:10B0E000A5113112BE124D13DE13701404159A15FA
:10B0F0003216CB16651701189F183E19DF19811AF1
:10B10000251BCA1B711C181DC21D6C1E181FC51FD4
:10B1100073202321D42186223923ED23A22458250C
:10B120000F26C82681273B28F628B2296F2A2D2B07
:10B13000EC2BAB2C6B2D2C2EED2EAF2F723035312E
:10B14000F931BD32823348340E35D4359B366237FF
:10B150002938F138B939813A493B123CDB3CA43DEE
:10B160006D3E363FFF3FC84091415A422343EB4377
:10B17000B4447C4545460C47D4479C486349294A1A
:10B18000F04AB64B7B4C404D044EC84E8C4F4E504F
:10B190001051D251935253531254D0548E554B5692
:10B1A0000757C2577C583659EE59A55A5C5B115C5B
:10B1B000C55C785D2A5EDB5E8A5F3960E66091611E
:10B1C0003C62E5628D633364D9647C651E66BF664C
:10B1D0005F67FC6798683369CC69646AF96A8E6B4B
:10B1E000206CB16C406DCD6D596EE26E6A6FF06F80
:10B1F0007570F7707871F6717372EE726673DD7345
:10B200005274C5743675A47511767B76E4764A77E8
:10B21000AE7710787078CE7829798379DA792F7AB9
:10B22000817AD27A207B6C7BB57BFC7B417C847CF1
:10B23000C47C027D3E7D777DAE7DE27D147E447EC2
:10B24000717E9C7EC47EEA7E0E7F2F7F4E7F6A7F5A
:10B25000847F9B7FB07FC37FD37FE17FEC7FF47FD0
:10B26000FB7FFE7FFF7F0000000000000000000069
:10B27000991700000000000000000000000000001E
:10B28000D9170000000000000000000000000000CE
:10B29000191900000000000000000000000000007C
:10B2A000F91C0000000000004E4F3A20756E6162EC
:10B2B0006C6520746F206F70656E2066696C650028
:10B2C0005945533A2061626C6520746F206F706538
:10B2D0006E2066696C6500FF000000000000000041
:10B2E000A51E0000BD1E00003D200000E91E00005C
:10B2F000151F00004D1F00000000000000000000AE
:10B3000079360000515900007C3C3E5E2B3D3F2FBA
:10B310005B5D3B2C2A225C00000000000000000066
:10B320000D3B0000113C0000513B0000653B00005C
:10B33000913B00004D3B0000050E08090D0C06076F
:10B340000F04001303931A9217C585848687C400DF
:10B350006FF07F030370037813F0800FFBD070470A
:10B360004008FE4340A004404408FE4344A004407B
:10B370000018FE4300C004403000FE4330900440FB
:10B380003400FE43349004401C18FE431CC00440AB
:10B390001018FE4310C004400818FE4308C00440C3
:10B3A0000C18FE430CC004400C10FE430CB00440CB
:10B3B0001010FE4310B004401810FE4318B00440B3
:10B3C0001C10FE431CB004401410FE4314B0044093
:10B3D0000418FE4304C004400010FE4300B00440C3
:10B3E0000008FE4300A004400408FE4304A00440FB
:10B3F0000C08FE430CA004400808FE4308A00440CB
:10B400001418FE4314C004401818FE4318C004402A
:10B410000410FE4304B004400810FE4308B004408A
:10B420001400FE43149004404C08FE434CA004401A
:10B430000420FE4304D004402410FE4324B0044002
:10B440002010FE4320B004402810FE4328B00440E2
:10B450002C10FE432CB004400020FE4300D00440DA
:10B460004808FE4348A004401000FE4310900440EA
:10B470000D0A0000FFFFFFFF0000000000000000B9
:10B48000555D0000615D0000355D00003D5D000020
:10B49000455D00004D5D000000151915000100001C
:10B4A000A88FFF1F1200000000020000D48FFF1FB2
:10B4B00043000000000300003090FF1F0000000068
:10B4C00001030904BC8FFF1F0000000002030904F0
:10B4D0001890FF1F00000000030309043490FF1FB1
:10B4E000000000000000000000000000000000005C
:10B4F00000000000000000007D700000957000005A
:10B500004D7000005D700000557000006570000017
:10B51000E16F0000F96F0000197000002170000059
:10B520002D7000003D7000006D700000757000000F
:10B53000B16F0000BD6F0000C96F0000D56F000043
:10B54000A5700000897000000000000000000000ED
:10B55000A9710000C17100007971000089710000BB
:10B5600081710000917100000D71000025710000D3
:10B57000457100004D7100005971000069710000B3
:10B5800099710000A1710000DD700000E9700000F9
:10B59000F570000001710000D1710000B57100006C
:10B5A0000000000000000000D5720000ED720000F5
:10B5B000A5720000B5720000AD720000BD720000FF
:10B5C000397200005172000071720000797200003F
:10B5D0008572000095720000C5720000CD720000F7
:10B5E0000972000015720000217200002D72000027
:10B5F000FD720000E1720000706F7700FFFFFFFF37
:10B6000000000000000000000000004003B8E23F1E
:10B61000000000000000000006D0CF43EBFD4C3ED0
:10B62000000000000000F03F000000000000F83FB4
:10B63000000000000000304300000000000030C3A4
:10B64000430000005090FF1F0020202020202020D9
:10B6500020202828282828202020202020202020C2
:10B6600020202020202020202088101010101010D2
:10B67000101010101010101010040404040404041E
:10B6800004040410101010101010414141414141B8
:10B69000010101010101010101010101010101019A
:10B6A00001010101101010101010424242424242AA
:10B6B000020202020202020202020202020202026A
:10B6C0000202020210101010200000000000000012
:10B6D000000000000000000000000000000000006A
:10B6E000000000000000000000000000000000005A
:10B6F000000000000000000000000000000000004A
:10B700000000000000000000000000000000000039
:10B710000000000000000000000000000000000029
:10B720000000000000000000000000000000000019
:10B730000000000000000000000000000000000009
:10B74000000000000000000000000000F8B500BF8D
:10B75000F8BC08BC9E467047E1AB00003504000011
:10B76000DD140000E1180000FD180000651B00005A
:10B77000811B00009D1B0000B91B0000112500006B
:10B78000312D0000953D0000715D0000C17000008A
:08B79000ED71000019730000C7
:04B79800F8B500BF41
:10B79C0000000000FA00000001010000D0070000CA
:10B7AC00010000000F000000010000000600000076
:10B7BC000100000002000000010000000300000076
:10B7CC000A00000028000000FFFFFFFF0A04000031
:10B7DC0094FFFF1FFFFFFFFF120100020200004059
:10B7EC00C016830400010102030100001803540079
:10B7FC00650065006E0073007900640075006900D7
:10B80C006E006F0009024300020100C032090400FF
:10B81C0000010202010005240010010524010101B0
:10B82C0004240206052406000107058203100040CB
:10B83C0009040100020A0000000705030240000091
:10B84C000705840240000000160355005300420017
:10B85C002000530065007200690061006C0000005C
:10B86C00040309040C0300000000000000000000A9
:10B87C0000000000000000000000000001000000BB
:10B88C00000000003C93FF1FA493FF1F0C94FF1FAC
:10B89C00000000000000000000000000000000009C
:10B8AC00000000000000000000000000000000008C
:10B8BC000000000040B60000000000000000000086
:10B8CC00000000000000000000000000000000006C
:10B8DC00000000000000000000000000000000005C
:10B8EC00000000000000000000000000000000004C
:10B8FC00000000000000000000000000000000003C
:10B90C00000000000000000000000000000000002B
:10B91C00000000000000000000000000000000001B
:10B92C00000000000000000001000000000000000A
:10B93C000E33CDAB34126DE6ECDE05000B000000CF
:10B94C0000000000000000000000000000000000EB
:10B95C0000000000000000000000000000000000DB
:10B96C0000000000000000000000000000000000CB
:10B97C0000000000000000000000000000000000BB
:10BCAC0000000000000000005090FF1F000000008A
:10BCBC00000000007C94FF1F7C94FF1F8494FF1FE6
:10BCCC008494FF1F8C94FF1F8C94FF1F9494FF1F70
:10BCDC009494FF1F9C94FF1F9C94FF1FA494FF1F20
:10BCEC00A494FF1FAC94FF1FAC94FF1FB494FF1FD0
:10BCFC00B494FF1FBC94FF1FBC94FF1FC494FF1F80
:10BD0C00C494FF1FCC94FF1FCC94FF1FD494FF1F2F
:10BD1C00D494FF1FDC94FF1FDC94FF1FE494FF1FDF
:10BD2C00E494FF1FEC94FF1FEC94FF1FF494FF1F8F
:10BD3C00F494FF1FFC94FF1FFC94FF1F0495FF1F3E
:10BD4C000495FF1F0C95FF1F0C95FF1F1495FF1FEB
:10BD5C001495FF1F1C95FF1F1C95FF1F2495FF1F9B
:10BD6C002495FF1F2C95FF1F2C95FF1F3495FF1F4B
:10BD7C003495FF1F3C95FF1F3C95FF1F4495FF1FFB
:10BD8C004495FF1F4C95FF1F4C95FF1F5495FF1FAB
:10BD9C005495FF1F5C95FF1F5C95FF1F6495FF1F5B
:10BDAC006495FF1F6C95FF1F6C95FF1F7495FF1F0B
:10BDBC007495FF1F7C95FF1F7C95FF1F8495FF1FBB
:10BDCC008495FF1F8C95FF1F8C95FF1F9495FF1F6B
:10BDDC009495FF1F9C95FF1F9C95FF1FA495FF1F1B
:10BDEC00A495FF1FAC95FF1FAC95FF1FB495FF1FCB
:10BDFC00B495FF1FBC95FF1FBC95FF1FC495FF1F7B
:10BE0C00C495FF1FCC95FF1FCC95FF1FD495FF1F2A
:10BE1C00D495FF1FDC95FF1FDC95FF1FE495FF1FDA
:10BE2C00E495FF1FEC95FF1FEC95FF1FF495FF1F8A
:10BE3C00F495FF1FFC95FF1FFC95FF1F0496FF1F39
:10BE4C000496FF1F0C96FF1F0C96FF1F1496FF1FE6
:10BE5C001496FF1F1C96FF1F1C96FF1F2496FF1F96
:10BE6C002496FF1F2C96FF1F2C96FF1F3496FF1F46
:10BE7C003496FF1F3C96FF1F3C96FF1F4496FF1FF6
:10BE8C004496FF1F4C96FF1F4C96FF1F5496FF1FA6
:10BE9C005496FF1F5C96FF1F5C96FF1F6496FF1F56
:10BEAC006496FF1F6C96FF1F6C96FF1F7496FF1F06
:10BEBC007496FF1F7C96FF1F7C96FF1F8496FF1FB6
:10BECC008496FF1F8C96FF1F8C96FF1F9496FF1F66
:10BEDC009496FF1F9C96FF1F9C96FF1FA496FF1F16
:10BEEC00A496FF1FAC96FF1FAC96FF1FB496FF1FC6
:10BEFC00B496FF1FBC96FF1FBC96FF1FC496FF1F76
:10BF0C00C496FF1FCC96FF1FCC96FF1FD496FF1F25
:10BF1C00D496FF1FDC96FF1FDC96FF1FE496FF1FD5
:10BF2C00E496FF1FEC96FF1FEC96FF1FF496FF1F85
:10BF3C00F496FF1FFC96FF1FFC96FF1F0497FF1F34
:10BF4C000497FF1F0C97FF1F0C97FF1F1497FF1FE1
:10BF5C001497FF1F1C97FF1F1C97FF1F2497FF1F91
:10BF6C002497FF1F2C97FF1F2C97FF1F3497FF1F41
:10BF7C003497FF1F3C97FF1F3C97FF1F4497FF1FF1
:10BF8C004497FF1F4C97FF1F4C97FF1F5497FF1FA1
:10BF9C005497FF1F5C97FF1F5C97FF1F6497FF1F51
:10BFAC006497FF1F6C97FF1F6C97FF1F7497FF1F01
:10BFBC007497FF1F7C97FF1F7C97FF1F8497FF1FB1
:10BFCC008497FF1F8C97FF1F8C97FF1F9497FF1F61
:10BFDC009497FF1F9C97FF1F9C97FF1FA497FF1F11
:10BFEC00A497FF1FAC97FF1FAC97FF1FB497FF1FC1
:10BFFC00B497FF1FBC97FF1FBC97FF1FC497FF1F71
:10C00C00C497FF1FCC97FF1FCC97FF1FD497FF1F20
:10C01C00D497FF1FDC97FF1FDC97FF1FE497FF1FD0
:10C02C00E497FF1FEC97FF1FEC97FF1FF497FF1F80
:10C03C00F497FF1FFC97FF1FFC97FF1F0498FF1F2F
:10C04C000498FF1F0C98FF1F0C98FF1F1498FF1FDC
:10C05C001498FF1F1C98FF1F1C98FF1F2498FF1F8C
:10C06C002498FF1F2C98FF1F2C98FF1F3498FF1F3C
:10C07C003498FF1F3C98FF1F3C98FF1F4498FF1FEC
:10C08C004498FF1F4C98FF1F4C98FF1F5498FF1F9C
:10C09C005498FF1F5C98FF1F5C98FF1F6498FF1F4C
:10C0AC006498FF1F6C98FF1F6C98FF1F7498FF1FFC
:10C0BC007498FF1F00000200FFFFFFFF48B600004E
:00000001FF
